:020000040800F2
:1030000000800020EFAB000895A00008B9A00008E0
:1030100000000000000000000000000000000000B0
:10302000000000000000000000000000C5B1000822
:103030000000000000000000C7B10008FD010020F2
:10304000C1AB0008C3AB0008C5AB0008C7AB0008A4
:10305000C9AB0008CBAB0008CDAB0008CFAB000874
:10306000D1AB000805020020D3AB0008D5AB0008A7
:1030700095020020D7AB0008D9AB0008DBAB0008F5
:10308000DDAB0008E1A00008F1A0000801A10008E4
:1030900011A1000821A1000831A10008DFAB000840
:1030A000E1AB0008E3AB0008E5AB0008F10200204B
:1030B000E7AB0008E9AB0008EBAB0008EDAB00089C
:1030C000014802490160704708ED00E00030000847
:1030D000B0B51E4D2C1F20688006400F411E0329ED
:1030E00022D81B487944097949008F442301171AD3
:1030F000296803220A40032A00D016482968490695
:10310000490F491C07F076FB29684904490E4843DA
:103110002968490F491C07F06DFB0BE07D20000278
:1031200008E00120C00305E00C3D28688004410F41
:103130000848C84008490860226892093C231340A7
:10314000064AD258D0400860B0BDC0460C100240BC
:1031500000127A000024F40070040020603100089E
:10316000000000000000000000000000000000005F
:10317000000000000000000000000000000000004F
:103180000100000002000000030000000400000035
:103190000600000007000000080000000900000011
:1031A000000000000000000000000000000000001F
:1031B0000100000002000000030000000400000005
:1031C00010B50124200207490A6802430A60022060
:1031D00000F00AF8002801D0012010BD06F03AFFE7
:0831E000002010BD0020024098
:1031E800B0B505460E4801780124002916D07D2087
:1031F800C00007F0FBFA01460A48006807F0F6FA33
:1032080000F0D6FD032D09D8002807D10024E0439B
:103218002946224600F082FD034805602046B0BDDD
:0C322800FA010020700400205C0400206B
:103234000348007803490A68101808607047C046BC
:08324400FA010020B81200207D
:0C324C00014800687047C046B81200201E
:10325800B0B50446FFF7F6FF0546601C02D00448E7
:1032680000780419FFF7EEFF401BA042FAD3B0BD67
:04327800FA01002037
:10327C0003490A6802239A4302430A607047C04616
:04328C0030000140CD
:1032900002480168012291430160704730000140FB
:1032A00003214902024A13688B43034313607047AA
:0432B00000000140D9
:1032B400F0B587B0044600200690002C60D005903D
:1032C400A06D002807D125465435204603F038FA6E
:1032D40000202870E06501273D072668B068C0001B
:1032E40012D4B068814901402943B1608048006824
:1032F400804907F07DFA4000801C0690069800285B
:1033040002D00698401EF8E7B068284208D1A06DA4
:1033140010210143A165E06D012105910843E06599
:10332400B06804210140A06D102210404018A16D26
:1033340029D1204620300F230393DB430193F33B31
:103344001940891CA165B168C90721D1F168182306
:103354009943A3680B43F36003218B0761680D460F
:103364001D40E76C2F43057F012D049313D1256C79
:103374002F43656C3D43A76C2F4301233B430BE074
:10338400012007B0F0BD1143A165384607B0F0BD78
:103394000021029118E03B463569574F2F400293B4
:1033A4001F4337610125EF07B9420DD0049B9942B1
:1033B4000AD0AB07994207D0039B9B0419404F4D99
:1033C4002F689F4379182960216B4B1E994109038B
:1033D400237E9B03657EEF031F43A57E6B033B4364
:1033E400E7681F430F4323690121002B00920491D6
:1033F40003DACA071946914300E049050F43017BEC
:1034040049003943007801280BD1002D029F0AD0CE
:10341400A06D20220243A265E06D01220243E26511
:1034240003E0029F01E000040143039D606A002859
:1034340005D00722920110400843A16A0143F068B5
:103444002F4A02400A43F26030692E4A02403A434E
:103454003261706907229043626B02437261706942
:1034640070229043A26B120102437261002B10D0B0
:103474000498400583421BD1206E00230246DA40A3
:103484002A400F2A03D01B1D202BF7D106E0042B62
:1034940004D1B06A019A1043B06209E0B26AE269E9
:1034A40092001C321C231340019A9A400243B262D8
:1034B400F068154A02408A420AD10020E065A06DF6
:1034C4000121014302208143A165059807B0F0BDA5
:1034D400A06D0099084302218843A065E06D04991A
:1034E4000843E065084607B0F0BDC046E8FFFF6F3B
:1034F40070040020400D030002FCFF1F0827014058
:0C3504001902FEFF02FCFFDFE7FF3F831F
:1035100070B50546006881680024490701D420463B
:1035200070BD8168890704D481680F4A0A4010324F
:103530008260FFF78BFE0646286880684007EED55C
:10354000FFF784FE811B28680329F6D381684907A9
:10355000F3D5A86D10210143A965E86D012420432E
:0C356000E865012070BDC046E8FFFF7F59
:10356C0070B505460068816882680024D20726D0B1
:10357C000222114023D1816805220A40012A16D16A
:10358C008168104A0A40911C816003210160FFF799
:10359C0057FE064628688068C00710D0FFF750FE1B
:1035AC00811B28680329F6D38168C907F3D0A86D5D
:1035BC0010210143A965E86D01242043E8652046EC
:0835CC0070BDC046E8FFFF7F5F
:1035D400F0B581B005460024009400688168C907ED
:1035E4001AD18168214A2F32114208D0A86D1021C6
:1035F4000143A965E86D01242043E8650CE0816876
:103604001A4A1140012739438160194800680002B1
:1036140005D4687E01280FD1204601B0F0BD1548BD
:103624000068154907F0E4F8401C00900098002851
:10363400EFD00098401EF8E7FFF706FE064628681C
:103644000168C907E8D18168C90704D18168074ABC
:10365400114039438160FFF7F7FD811B2868032976
:10366400EED30168C907EBD1C0E7C046E8FFFF7F8E
:0C3674000827014070040020400D0300F6
:10368000F0B581B00E46044601688B6802205B07E6
:103690001BD400925422A25C012A16D0274654372C
:1036A00001253D70C868C0070AD18868C00704D0EA
:1036B0008868194A0240901C8860C8682843C8601E
:1036C0002046FFF787FF002801D001B0F0BDA06DB4
:1036D0001249014028020818A0650020E065216811
:1036E0001C220A603870206D0D4A0E4B0E4DC562CB
:1036F000036342634A68102313434B6040313246F0
:10370000009B00F023FD21688A68034B13401A1DBB
:103710008A6001B0F0BDC046E8FFFF7FFEF0FFFF0A
:0C372000FFAB0008F5AB000893B30008F5
:10372C00F0B589B0002508955422825C012A01D19C
:10373C000224DCE006465436012434700268936897
:10374C005B0711D404694B68022B12D1042004438B
:10375C008148844252D17F48C0430B68D94301430E
:10376C00906A084090624AE0816D20220A4382658B
:10377C00BCE00796069304263443764B764FBC4246
:10378C004DD10F683B40906A1843906238025369E0
:10379C0083438968014071480840184350610024F4
:1037AC00002F01D4079EA1E001266D483B46076817
:1037BC0007208205394611406A48029383426CD136
:1037CC00F0053B46034068D1654F3B689343194372
:1037DC000143396066480068664907F005F80C211A
:1037EC0041430C31089108980028DBD0079E0898BB
:1037FC00401E089008980028F9D177E00B68002447
:10380C00002B73D556480168574A934262D0574AE9
:10381C00934262D0534A934268D105225BE00296F0
:10382C0005951F27069C27400F2500950397BD4043
:10383C00046E0195AC4304940F681F4246D0FB07FD
:10384C00059D2C465BD1BB0754D47B0754D43B0756
:10385C0054D4FB06344652D4BB0663D47B0663D4E3
:10386C003B0663D4FB0563D40297BB0562D47B058E
:10387C0062D43B0562D4FB0462D4BB0462D47B04E7
:10388C0062D43B04009C3AD4FB035FD4BB035FD4EB
:10389C007B03DB1712241C4031E03348029B83422C
:1038AC0003D130063B46034008D03048029B83428C
:1038BC0000D077E7B005074000D073E7284F3B688E
:1038CC009343194301433960079E0FE07B00DC0EE4
:1038DC00059D14E00322920501E00322D20511405C
:1038EC0007229205036893435918016035702046EE
:1038FC0009B0F0BD012402E0022400E00324039E81
:10390C00B440049B1C430466069B9B08C069984208
:10391C0000D83BE70198C043936A0340B800000FFE
:10392C00B04031E70524EAE70624E8E70724E6E798
:10393C000824E4E70924E2E70A24E0E70B24DEE7A5
:10394C000C24DCE70D24DAE70E24D8E71024D6E7A4
:10395C001124D4E7FFFF07000400008000FFFF07DD
:10396C0008270140001000B0004000B8002000B44F
:08397C0070040020400D03005F
:10398400F0B582B05422825C012A01D102212AE1DD
:10399400026893685B07B44E00D504E190C9083906
:1039A400B44213D10124E505AF4260D00325AD052F
:1039B400AF4264D11F26B6068F683740D668AF4B36
:1039C4003340A94EFB185B19D3605CE00126F30574
:1039D4009F425ED00325AB059F426AD11346A033B4
:1039E40000938B68A44F01931F40A04B9C426DD160
:1039F400002F00D1A7E0019CE30700D0ABE0A307B0
:103A040000D5A9E0630700D5F0E0230700D5F1E075
:103A1400E30600D5F0E0A30600D5F1E0630600D587
:103A2400F2E0230600D5F3E0E30500D5F4E0A305B6
:103A340000D5F5E0630500D5F6E0230500D5F7E0F1
:103A4400E30400D5F8E0A30400D5F9E0630400D54D
:103A5400FAE0230400D5FBE0E30300D5FCE0A30374
:103A640000D5FDE06303DB1712261E4074E0D36823
:103A74003746824E1E4073193E46D36003E0D36836
:103A84007E4D1D40D5602304846D9C438465802451
:103A940080E0774BDB43E5431D43E30C04261E40E3
:103AA4009319A0269F592F40724D25403D439D51A7
:103AB4005FE06F4BDB43E5431D43E30C04241C40F0
:103AC4001319A0241E592E401E5152E0002F3ED03F
:103AD400019FFB0747D1BB07344645D47B0700D57C
:103AE40086E03B072C463FD4FB0600D586E0BB06A8
:103AF40000D587E07B0600D588E03B0600D589E049
:103B0400FB0500D58AE0BB0500D58BE07B0500D51D
:103B14008CE03B0500D58DE0FB0400D58EE0BB04B2
:103B240000D58FE07B0400D590E03B0400D591E004
:103B3400FB0300D592E0BB0300D593E07B03DB17C6
:103B440012241C4010E0019B5B00DE0E04E0019B8C
:103B54005B00DC0E08E000260123B340009D2C68C6
:103B64001C432C6005E00024A640009C636833439A
:103B74006360846D0B683D4DAB423B4E05D1012320
:103B84005D04AC4384651C0204E001239D04AC4342
:103B940084655C02146055680B7B012B01D12543BD
:103BA40000E0A543556054300D690C68B4420AD155
:103BB400D3689B08062633409D40D3689F0837404E
:103BC4004B69BB4000E04B69002101702804184395
:103BD400A302DC0F9B0F1B199B00D218136A284CFD
:103BE4001C4004431462084602B0F0BD0226B3E749
:103BF4000224B9E70326AFE70426ADE70424B3E7BC
:103C04000526A9E70524AFE70626A5E70624ABE7C2
:103C14000726A1E70724A7E708269DE70824A3E7CA
:103C2400092699E709249FE70A2695E70A249BE7D2
:103C34000B2691E70B2497E70C268DE70C2493E7DA
:103C44000D2689E70D248FE70E2685E70E248BE7E2
:103C54000F2681E70F2487E710267DE7102483E7EA
:103C6400112679E711247FE70000C07CFFFF1700CD
:103C7400FFFFC77CFFFF8700FFFF0700FFFF3F83B5
:043C840000F000F05C
:103C8800F0B583B00446002602965420205C012833
:103C980001D102253CE02746543701253D702046D6
:103CA800FFF760FC21688A68D207A26D21D10090D5
:103CB80081235B009A43921CA265CA68CB680320E3
:103CC80001908343CB60EB078868184388600198AC
:103CD8000240114B886800280FD50298401C0290BA
:103CE80002989842F6D3A06D102202430220824324
:103CF8000CE010210A43054608E0C8681043C86074
:103D0800A06D0122024302208243009D3E70A265FD
:0C3D1800284603B0F0BDC04600F20200D7
:103D2400002805D40322034693430C4A9A1806E05C
:103D34000F220240083A03239A43074BD218800704
:103D4400C00E8901C9B28140FF23834010689843A3
:103D5400084310607047C0461CED00E000E400E03A
:103D6400002805D41F210840012181400148016039
:083D74007047C04600E100E0C9
:103D7C00002809D41F21084001218140034801601B
:103D8C00BFF34F8FBFF36F8F7047C04680E100E0E9
:103D9C00BFF34F8F034804490160BFF34F8F00BF3F
:0C3DAC00FDE7C0460CED00E00400FA0545
:103DB800401E010E01D0012070470749074A506094
:103DC800074803680B400321890759180160002040
:103DD8009060072111607047FFFFFF0010E000E0CE
:043DE80020ED00E0EA
:103DEC00B0B5002813D00446407F002803D12077BB
:103DFC00204602F01FFD022060772079002808D0B1
:103E0C00A168E268204600F027F8002808D00120BD
:103E1C00B0BD20680F4941618168182291438160CF
:103E2C0000256079002801D0216900E0E943206871
:103E3C00016181686022914362690A4382608168F2
:103E4C0080229143A2690A4382600120607700209E
:083E5C00B0BDC046B71DC10452
:103E6400F0B51F250024002D07D06D1E1F232B4005
:103E74000E46DE40F307F5D000E0E5430323164683
:103E8400DE410123032E0FD87E4436797600B744F1
:103E940003010D100F2D07D80068416181681823B4
:103EA40099431143816000231846F0BD072DF3D9CF
:083EB400FAE7062DF0D9F7E74B
:103EBC00F0B581B004464079012802D1022001B04E
:103ECC00F0BD15460E460220207101276771086867
:103EDC00042840D1002D08D02068406B002819D54B
:103EEC00FFF7AEF90228F7D30CE00097FFF7A8F91B
:103EFC0007462068406B000414D5FFF7A1F9C01BDE
:103F0C000228F6D320690821014321610320207186
:103F1C0001B0F0BD00970120FFF798F92068B16956
:103F2C00416405E00120FFF791F92068B169016453
:103F3C0010212940F2698A40214B8B40876C9F43AA
:103F4C0017438764326A8A40FF238B40C16C9943C4
:103F5C001143C164009F2068316901290AD11021E5
:103F6C000D407169A9401F22AA40836B93430B43F8
:103F7C00836301E010210D400721A940C26B8A43E5
:103F8C003168B3680B43F1681943A9401143C1630D
:103F9C00B903A94002688A4302607168A940094AC2
:103FAC00AA40036893430B430360C021A9400268F5
:103FBC008A43026000206071277101B0F0BDC046D9
:083FCC00FF030000FE0F0000DE
:103FD400F0B583B000283FD00446064624360220BC
:103FE4007070276838683049014039602F48803044
:103FF400A0642F483818142106F0FAFB80002B49DE
:104004004118206401916164F8B20838142106F063
:10401400EFFB1F210140012528468840E064A26887
:10402400E168114323690B4361691943A3690B4395
:10403400E1691943236A0B433968194339600295CE
:10404400A9038A421B4A0AD1002301990B606360C9
:1040540010601F461D461CE0012003B0F0BD6368DC
:104064003F211940019D29601060581E0023032838
:104074001F461D460DD8481E810053180021D967DC
:1040840003210140029D8D400B4805607C33BC3206
:1040940017460020E06323656765A56530700299C3
:1040A400717003B0F0BDC0460F80FFFF00080240EE
:0C40B400F8FFFDBF8408024044090240F0
:1040C000F0B581B004462420205C012802D10220F2
:1040D00001B0F0BD25462435012028706E78012EF0
:1040E0002CD1022068700020E06325682F680096BC
:1040F000B7432F60A76CE66C7E60266D002E02D061
:10410000666DA76D7760266C1C273740009EBE4009
:104110000D4F3F6837430C4E37606B60A368102B20
:10412000144600D00C46AC60102B00D01146E9605C
:104130002968009A1143296001B0F0BD002129705F
:0C4140008021E16301B0F0BD04000240EA
:10414C00F0B582B004462420205C012802D1022064
:10415C0002B0F0BD174625462435012028706A7838
:10416C00012A2ED1022068700020E06325682A689D
:10417C0001260196B2432A60A26CE66C5660226D51
:10418C000092002A02D0626DA66D5660226C1C262D
:10419C001640019AB2401C4E366816431A4A1660F5
:1041AC006B60A368102B3A4600D00A46AA60102B0D
:1041BC0000D03946E9602968226B002A07D00E220C
:1041CC000AE0002129708021E16302B0F0BD0422D5
:1041DC00914329602A680A21114329600199090237
:1041EC00626C1368DB0302D513680B431360009BEE
:1041FC00002B02D01A680A431A602968019A1143ED
:0C420C00296002B0F0BDC0460400024072
:1042180070B500282AD0014624314A78022A27D1CD
:10422800046822680E239A432260426C1568134B77
:104238001D4015602568012295432560046C1C25E6
:1042480025401446AC400E4D2E6826432E60846CE3
:10425800C56C6560046D002C05D025681D4025607F
:10426800436D806D58604A70002004E0012070BDE5
:104278000422C263012000220A7070BDFFFEFFFF06
:0442880004000240EC
:10428C00F0B585B00446054624356878022809D176
:10429C002068006880060CD41646002901910DD0C8
:1042AC0004220CE0002028700420E063012005B0FB
:1042BC00F0BD01200102E16305B0F0BD0222206CCB
:1042CC001C2104910840824003923348071FFEF7DB
:1042DC00B7FF039A02903868104217D1216C0498EA
:1042EC0001403868C840000748D4701CF3D0FEF772
:1042FC00A7FF039A002E03D00299401AB042EAD9C4
:10430C002020E06300202870012041E0206D00286F
:10431C000ED0616DA26D0B681A4209D001231E02EA
:10432C000768374307604A609802E16B0143E16319
:10433C00A06CE16C0268114205D041600120400282
:10434C00E16B0143E163206C049908400199002959
:10435C0008D004218140104A1068084310600020E6
:10436C0005B0F0BD022181400B4A10680843106073
:10437C00002028700121697005B0F0BD01200246B3
:10438C008A40054B196811431960E06300212970BC
:0C439C00687005B0F0BDC046040002408F
:1043A800F0B585B00E46234D2978012902D10220A7
:1043B80005B0F0BD17460193049000246C600120FD
:1043C800039028707D20C000029000F037F8002884
:1043D8002DD10399029B0094174D0498012809D107
:1043E8002868084328603760BFF36F8F01987060B2
:1043F800184614E08804296801432960EFF3108403
:1044080072B6009904CF04C64A1C3F291146F9D355
:104418001846291F0968C903FBD484F3108800F0E3
:104428000DF82968049A91432960024D009C2C706C
:0C44380005B0F0BD3C1200201420024032
:1044440070B50446FEF700FF0619104D2868C00336
:1044540005D5FEF7F9FEB042F8D3032070BD2868F5
:104464000B494A1C2A60084003D00A4948600120CD
:1044740070BDFEF7E9FE04192868400304D5FEF771
:10448400E3FEA042F8D3E8E7002070BD102002400C
:08449400FAC300003C120020F5
:10449C000648C168002901D4002070470449016016
:1044AC0004490160C068C00F7047C0460820024034
:0844BC0023016745AB89EFCD38
:1044C4000120C00703490A6802430A600868C04320
:0844D400C00F704714200240E4
:1044DC00F0B583B00546284C2078012802D1022083
:1044EC0003B0F0BD029100276760012020707D2091
:1044FC00C6003046FFF7A0FF002839D104206860C1
:10450C002868042809D11E48801C1C490A680243EB
:10451C000A603046FFF790FF2AE0F84302990860E2
:10452C000021AF68E868C01987420191084619D28A
:10453C00FC0012490868134A10402043104A1043EB
:10454C0008603046FFF778FF002808D1A868E968B2
:10455C00081808347F1C8742EBD3019801E00299BC
:10456C000F60054C054B1968022291431960019F9D
:10457C00277003B0F0BDC0463C120020142002404E
:08458C000200010005FEFEFF24
:10459400F0B58AB00C68002C00D1C1E00246614835
:1045A400824201D0052000E00320009000231E4633
:1045B400099308930691049211E03043079E5A4CE4
:1045C40060605B1C0C682046D840089D2D1D089532
:1045D4000836099DAD1C0995002800D1A0E00125ED
:1045E40003959D402C400594EBD0099A07964F689B
:1045F400032408463E462640711E0129029714D81A
:10460400019313469440049A9168A143C06898406A
:1046140008439060F806019BC00F98405168A94375
:1046240001435160E5435F0008E0032017469040D2
:10463400C543032E049A01D1099C23E0D068284085
:104644001446069A9168B9400143E160022E3C4643
:1046540017D11C20089908400F2181400294DC08DE
:10466400A400049F3C192E46256A8D43116981409C
:10467400294335462162029C516803260E403A467E
:1046840001E0049A0299A640106828403043106063
:104694008803800F0699079E93D0182131400F207C
:1046A400884003241D46A5431F4C6619356E854377
:1046B40060360520000782420CD01D48824206D095
:1046C4001C4882420098194A06D1022004E0174A85
:1046D400039801E00020154A8840284330601068A0
:1046E40006994D68EC0302D5059E304301E0059E12
:1046F400B04310605068AC0301D5304300E0B043D0
:10470400506009480068EC0201D5304300E0B04332
:10471400054A10605068AA0200D54EE7B0434DE741
:104724000AB0F0BD000C005000180240801802408E
:084734000004005000080050D1
:10473C00F0B58AB00290002972D03A48029A8242AF
:10474C0001D0052000E003200090002422462746DB
:10475C002646019125E0069D099885400868284366
:10476C0008601C20089C2040059B8340F0088000BA
:10477C0008180A46016A994301629068A843906040
:10478C005068079988435060D068A843D060099A54
:10479C000199761C0846F040241D921C083700280D
:1047AC003ED001231846B04005460D40F1D007908D
:1047BC000992089418243C400F210591A140032034
:1047CC00324606908243184880180390026E04917A
:1047DC000A40052000070299814208D01448814202
:1047EC0006D014488142009B02D1022300E0002332
:1047FC00A3409A42AFD1039B60330C4A1068A84384
:10480C0010605068A8435060074A1068A8431060B5
:10481C005068A84350601868049A904318609AE74F
:10482C000AB0F0BD000C0050001802408018024085
:08483C000004005000080050C8
:10484400F0B581B0032569020F4E32688A430243F2
:10485400326001214A020024904212D10B480268BE
:10486400706940050DD58F0206205043084905F0B4
:10487400BFFF801C401E03D071693942FAD100E0A9
:104884002C46204601B0F0BD0070004070040020AA
:0448940040420F008F
:10489800F0B587B00125002800D1EFE10495059017
:1048A8000078C007FD4F2AD0B868F96803252A4662
:1048B8008A43382101401020484082185042504114
:1048C800082914D0002812D1059842680120010453
:1048D8008A4208D005231B049A4200D028E18204AA
:1048E8003B6813433B603A680A433A6029E13868F9
:1048F800800304D505984068002800D188E0059811
:10490800007880073CD405980078000768D4059A99
:104918001078400771D4D06900282FD0B9683822A0
:104928000A40102A00D0DBE0012871D0F868032182
:104938000140059B1A6A91426AD1702101405A6A66
:10494800914265D17F21090201409A6A120291427F
:104958005ED11F2149040140DA6A914258D10721EA
:104968004A0602401C461B6B9A42049D00D085E112
:1049780049070840616B884200D07FE100257DE14E
:10498800B9683820084010214140FA6803263240AF
:1049980002235340CA18514251410125AC02002854
:1049A80038D0002936D13868059AD168002900D155
:1049B800D5E00721C90288431169014339602802FB
:1049C800396801433960FEF73DFC054638682042E6
:1049D80000D0D5E0FEF736FC401B0228F6D9CDE022
:1049E800B8683821014018293CD1386E80078ED527
:1049F8000598806900288AD10AE0B8683821014002
:104A0800202946D1F86D800785D59068002882D185
:104A1800049D33E139682142059B03D0D9680029F8
:104A280000D12BE17F2109027A688A43596909027A
:104A38001143796000280DD10720C00239688143ED
:104A480018690843386038688004400F9949C140A4
:104A58009948016099480068FEF7C2FB002800D019
:104A68000CE150E7386E05998969002900D1A7E063
:104A7800012108433866FEF7E5FB0646386E8007D5
:104A880000D544E7FEF7DEFB801B03250228F5D995
:104A9800F4E0012003900107F86B0840029006D16A
:104AA800F86B0843F863F86B084006900698019184
:104AB80083480068C0052AD403980402804908681E
:104AC80020430860FEF7BEFB06467D48006820428A
:104AD8001DD1FEF7B7FB801B03250228F5D9CDE0D1
:104AE80001221306396899433960022852D1039389
:104AF80004925406FEF7A6FB0646386820427ED08C
:104B0800FEF7A0FB801B03250228F6D9B6E005981E
:104B180080686C4C012806D0052800D098E0F86D14
:104B280004210143F965F86D03990843F86599E094
:104B38003B688B433B6081043B688B433B60002AA6
:104B48004FD04404FEF77EFB06463868204200D06A
:104B5800D5E6FEF777FB801B6428F6D98EE029029C
:104B680088433860FEF76EFB05463868204200D15E
:104B7800C9E6FEF767FB401B0228F6D935467DE0FB
:104B88007F20000279688143059840690002084344
:104B98007860B8E6F8680325A843F860F8684A49D9
:104BA8000140F9605606FEF74DFB0446386830426E
:104BB80000D1E3E6FEF746FB001B0228F6D95DE0CC
:104BC800012188433866FEF73DFB0646386E8007AC
:104BD80000D49CE6FEF736FB801B03250228F5D996
:104BE8004CE04404FEF72EFB06463868204200D10C
:104BF80085E6FEF727FB801B6428F6D93EE0F868B7
:104C080032490140059A106A0843516A0143906A83
:104C180000020843D16A0143106B526B08431043EA
:104C2800F860386803990843386004980007F96801
:104C38000143F960FEF706FB06463868204200D0BB
:104C48009CE6FEF7FFFA801B03250228F5D915E03C
:104C5800F96D039A9143F965F96D04229143F96559
:104C680000280ED0FEF7EEFA0646F86D800717D436
:104C7800FEF7E8FA801B0325A042F6D9284607B0BC
:104C8800F0BDFEF7DFFA0646F86D800708D5FEF797
:104C9800D9FA801B0325A042F6D9EFE7001002409D
:104CA80002980028059A00D035E6F86B01998843E8
:104CB800F86330E60024F400700400205C0400204F
:104CC8000070004088130000FFFFFEEE8C80C111C9
:104CD800F0B583B00D460121002800D1A3E0019171
:104CE80002905248006807242040A84213D24F4936
:104CF8000868A043284308604D4EFEF7A3FA07460C
:104D08004A4800682040A84205D0FEF79BFAC01B1D
:104D1800B042F5D986E0029B18688107454E0CD54C
:104D2800410703D5210332680A4332600F21090283
:104D380032688A43996811433160C00718D13B48EB
:104D480000682040A84228D938490868A043284369
:104D58000860374FFEF776FA064634480068204068
:104D6800A8421AD0FEF76EFA801BB842F5D959E06E
:104D7800586803282FD8810001A2515832468F461F
:104D8800994D0008E54D0008EF4D0008F94D000861
:104D980011460839096849052CE0029A107840073D
:104DA800244D05D5200329688143D068084328602D
:104DB80000F048F8296889093C220A401E498958A8
:104DC8001F220A40D0401D4908601D480068FEF7B0
:104DD80007FA014627E03246516D0AE011460839C4
:104DE8000968890306E0114608390968890101E064
:104DF800916D8907019916D51168A1430143116086
:104E08000B4FFEF71FFA06460A4800683821014092
:104E180002984068C000814291D0FEF713FA801BC7
:104E2800B842F1D90321084603B0F0BD0020024082
:104E38008813000008100240603100087004002048
:044E48005C040020E6
:104E4C0010B51E4C20688006400F06D02068382113
:104E5C00084008281A4807D110BD083C2068800477
:104E6C00410F1848C84010BD22680A40102A15D1BD
:104E7C00616803220A40032A00D01248616849067F
:104E8C00490F491C05F0B0FC61684904490E4843C0
:104E9C006168490F491C05F0A7FC10BD206808404B
:104EAC00202802D10120C00310BD2068084018281A
:104EBC0001D0002010BD7D20000210BD0810024062
:084ECC0000127A000024F4003A
:104ED4000648006806490968890A1C220A400549EF
:104EE40089581F220A40D0407047C04670040020F1
:084EF40008100240A031000883
:104EFC000120C00402490A6802430A607047C04698
:044F0C00001002404F
:104F100010B50320000208490C6820404860E005F5
:104F200002D4A00504D410BD05F00AFFA005FAD5EF
:0C4F300005F007FF10BDC0461C10024039
:104F3C00F0B587B0817889077A4F01D400264EE00E
:104F4C000590012319073A46183A10680840049056
:104F5C0006D1106808431060106808400690069847
:104F6C000292039101931E026F4C20683043206023
:104F7C00FEF766F905462068304207D1FEF760F966
:104F8C00401B0228F7D90326059820E0032005468C
:104F9C000102B868084012D00599096B88420BD001
:104FAC00B86801990904BA680A43BA60BA688A43B6
:104FBC00BA605E490840B860C00700D0A1E0BA688A
:104FCC005A4802400598016B1143B96000260499B8
:104FDC00002904D1029B1968039A91431960056852
:104FEC00E90762D1A90768D4E9066ED4A90575D47E
:104FFC0069057CD4A90606D5032109033A688A43BE
:10500C0001691143396001216A040ED53A68494B94
:10501C001A40046A22433A605A1C944205D10A048D
:10502C003B46483B1C6814431C602A0305D53A6870
:10503C0040239A43436A13433B608A05AB0211D564
:10504C003B689343846A23433B6094420AD10B062A
:10505C0004933C46483C0590304626681E43266027
:10506C000646059815420CD00A063B689343C46A61
:10507C0023433B60944204D13B46483B1C68144399
:10508C001C602A050ED58C03032292033B689343C4
:10509C00426913433B60A24204D10804483F39687B
:1050AC0001433960304607B0F0BD396803229143A3
:1050BC0042680A433A60A90796D539680C22914395
:1050CC0082680A433A60E90690D5032189023A685E
:1050DC008A43C16811433960A90589D50321890424
:1050EC003A688A43816911433960690582D5032185
:1050FC0009053A688A43C16911433960A90682D50A
:10510C007AE7FEF79DF80646094CB868800700D58B
:10511C0055E7FEF795F8801BA042F6D905982E4668
:10512C0055E7C0465410024000700040FFFCFFFFE2
:08513C0088130000FFFFFF3F94
:1051440030B5056801229407A04205D0234B98424C
:1051540002D0234B984204D170239D434B682B43C8
:1051640000E02B461F4DA84209DD1F4CA0420FDC76
:105174001A4CA04212D01F4CA0420FD02BE0A042E8
:105184000CD0174CA04209D01B4CA04206D022E000
:10519400164CA04202D0164CA0421CD10324240277
:1051A400A343CC681C4380239C434B692343036083
:1051B4008B68C3620B688362104BC3180A24E341F3
:1051C400072B06D814469C40E1231C4201D00969F0
:1051D4000163426130BD1C46E5E7C046002C014036
:1051E40000040040FF2B0140FF4301400048014000
:1051F40000440140004001400020004000D4FEBFB4
:105204003D21415C01290FD101463D3102220A7042
:1052140001681148814209DC0120800781420BD0DA
:105224001048814208D011E0012070470B488142A8
:1052340002D00B48814209D188680B4A0240002001
:10524400062A08D001231B049A4204D008680122CC
:1052540002430A6000207047FF2B014000400140D8
:0C526400002C0140000400400700010085
:1052700010B53D21415C012912D101463D31022288
:105280000A700168C86801221043C8600F48814253
:1052900008DC900781420BD00F48814208D010E013
:1052A000012010BD0A48814202D00A48814208D13B
:1052B00088680A4B03400020062B06D01404A34242
:1052C00003D0086810430860002010BDFF2B014088
:1052D00000400140002C0140000400400700010094
:1052E00010B50268D36801218B43D360136A074C61
:1052F000234206D1136A064C234202D113688B4322
:1053000013603D228154002010BDC04611110000E1
:045310004404000051
:10531400B0B50446006801698907554D17D5C168C1
:10532400890714D52946FE3101610121217780695D
:10533400800703D0204605F02EFD05E0204605F049
:105344002BFD204605F029FD002020772068016907
:10535400490718D5C168490715D52946FC310161AB
:105364000221217780698005800F03D0204605F053
:1053740012FD05E0204605F00FFD204605F00DFD69
:105384000020207720680169090717D5C16809073B
:1053940014D52946F831016104212177C0698007B9
:1053A40003D0204605F0F7FC05E0204605F0F4FCA8
:1053B400204605F0F2FC0020207720680169C90628
:1053C40018D5C168C90615D52946F03101610821EF
:1053D4002177C0698005800F03D0204605F0DBFCEF
:1053E40005E0204605F0D8FC204605F0D6FC002058
:1053F400207720680169C90709D0C168C90706D0A8
:105404002946FF310161204604F098FE20680169B5
:10541400090609D5C168090606D529468031016106
:10542400204605F0BDFC20680169C90507D5C1689F
:10543400090604D50561204605F0B3FC206801691E
:10544400490609D5C168490606D52946C031016116
:10545400204605F0A3FC20680169890607D5C168C8
:10546400890604D5E0350561204605F098FCB0BDF9
:04547400FFFEFFFF39
:1054780070B53C22825C012A01D1022070BD02462F
:105488003C320223537000688368474C1C40846098
:105498000B683F2B19DD5F2B1EDD602B41D00124EB
:1054A8006503AB4255D0702B79D1FF231B0284686A
:1054B8009C434B688D68C9681D43090229432143F1
:1054C800816083687721194368E01F2B1EDC002B5D
:1054D80020D0102B1ED062E0402B4AD0502B5ED13A
:1054E800036A046A0125AC4304628469F025AC436D
:1054F800CD682D01254385610A24A34349681943D2
:105508000162836829491940573147E0202B01D0AF
:10551800302B44D18168254C0C4023430721194383
:105528003CE0036A1024A34303620F231B0384692E
:105538009C43CB681B032343046A8361A0239C43D9
:105548004968090121430162836818491940673194
:1055580024E0FF231B0285689D434B688E68C96859
:105568001E430902314329438160A303816819431B
:1055780014E0036A046A0125AC4304628469F025D7
:10558800AC43CD682D01254385610A24A3434968AE
:105598001943016283680549194047318160002039
:1055A80010700121517070BD8800CEFF88FFCFFFB9
:1055B80070B53C22825C012A01D1022070BD0246EE
:1055C8003C3202235370006845688368134CA0423C
:1055D80001D02E4604E00F263605B5434E682E430B
:1055E8007025AE430D68354345600D4DA84205DC76
:1055F8000124A407A04206D00B4C02E0094DA842A2
:1056080001D0A04204D18024A34389681943816052
:10561800002010700121517070BDC046002C01405F
:0C562800FF2B0140004001400004004046
:10563400F0B581B004460268106871490140A06861
:105644002369034360691843E369184308431060FE
:105654000327380351688143E06808435060A16917
:10566400684DAA4202D0206A084300E008469168C7
:10567400654E0E4006439660D06A0F218843616AE6
:105684000843D0620026614882420EDD60488242AF
:105694001DD0AA4211D05F4882420CD160480068F4
:1056A4008007000F5F4E365811E05B48824208D0F5
:1056B4005A4882420BD0102609E059480068000A73
:1056C40001E0574800680C26064056488659204693
:1056D400683000905448AA4214D00125EA0393424A
:1056E40022D1082E00D981E07E4436797600B74471
:1056F400047D547D4D7D7D7D5300FFF7E9FB00283B
:1057040048D172E00125082E00D96FE07E44367935
:105714007600B744046B216B196B6B6B1F00FFF7AA
:10572400D7FB002814D160E0082E5FD87E44367978
:105734007600B744045B4B5B445B5B5B4A00FFF75A
:10574400C7FB00283FD150E0FFF77EFB00284CD078
:10575400616A01E00120C0034900344A515A05F04E
:1057640047F862685743B84240D3110388423DD892
:10577400010E5608000200238019594105F05CF817
:105784002C4941182C4A91422DD32FE0FFF75CFBA2
:1057940000282AD0616A00E010464900234A515A81
:1057A40005F026F8400061684A08101805F020F852
:1057B4001F4901401AD00007400F084313E0FFF7C8
:1057C40043FB002811D0616A00E010464900174AE3
:1057D400515A05F00DF861684A08101805F008F8E8
:1057E40080B2102802D32168C860002513480099AC
:1057F4000860002020676067284601B0F0BDC046FD
:10580400F369FFCF00800040FFF4FF11FF4B00401D
:10581400004C004000380140004400400048004073
:105824005410024014AB00080024F400E6B500084C
:10583400F0FF000000FDFFFF00FD0F00010001006C
:10584400F0B581B00546074680370024FC60FDF7BB
:10585400FBFC06462868016809070BD5114800902F
:105864000120410500222846334605F004FB0028A8
:105874000ED12868006840070CD50A480090012022
:10588400810500222846334605F0F5FA002801D0A8
:10589400032404E020207860B8603C70EC66204665
:0858A40001B0F0BDFFFFFF01A0
:1058AC00F0B581B005460446803460680223202898
:1058BC0011D10120002950D0002A4ED0AE680090A2
:1058CC000703BE420AD1C80708D02869002805D1B1
:1058DC00009801B0F0BD022001B0F0BD2078012885
:1058EC0018463AD02B4654335A800020E0601A8078
:1058FC00296521216160009B59076A6E8A4206D195
:10590C00BE4202D12869002808D0184907E0BE42DF
:10591C0002D12969002912D0124911E01249002044
:10592C0020706967EFF3108183F31088DA052B6818
:10593C009C6814439C6081F3108801B0F0BD084949
:10594C0020706967EFF3108183F310882A6813685D
:10595C0080241C43146081F3108801B0F0BDC04654
:10596C00F5590008CFB400087D59000863B400084D
:10597C0070B58421415821291AD1014656318A8AA1
:10598C00002A15D0174B02E0521E140410D00C88BC
:10599C00002C0ED00468E5692D06F5D5056D2E8812
:1059AC001E40A662AC1C04650C88641E0C80EBE7E0
:1059BC0070BDEFF31081012282F31088D3050468C7
:1059CC00A5689D43A56081F31088EFF3108182F3E5
:1059DC0010880068026840231343036081F3108829
:0859EC0070BDC046FF01000080
:1059F40030B58421415821290FD1014656310A88F6
:105A0400002A0BD0026D1388104C1C4003689C6262
:105A1400921C02650888401E088030BDEFF3108197
:105A2400012282F3108803681C688025AC431C6043
:105A340081F31088EFF3108182F310880068026804
:105A440040231343036081F3108830BDFF0100003D
:105A5400F0B581B0034680339C680226202C10D117
:105A6400012400290ED0002A0CD001252C038768BC
:105A7400A7420AD1CC0708D00469002C05D101241F
:105A840000E00224204601B0F0BD1C78012C34460D
:105A9400F8D00024C4661D7003680A4EB3420DD0CA
:105AA4005B681B020AD5EFF3108385F31088AD06FB
:105AB400066837682F43376083F3108800F004F8D2
:085AC400E0E7C046008000404D
:105ACC00F0B582B05C23C2528165002101670446A7
:105ADC005C346280856803468033002D0BD0012630
:105AEC003707BD420CD03603B5420ED10569002DE7
:105AFC0004D1334D0CE00569002D08D1FF2507E0DA
:105B0C000569002D03D03F2502E0A18001E07F252F
:105B1C00A5800191D96022259D60EFF310860125A7
:105B2C0085F310880768B9682943B96086F3108833
:105B3C00290200912F036907466E8E4202D1A1897A
:105B4C00914216D98168B94202D10169002933D03A
:105B5C001F4A0199009C19700267EFF3108185F3BD
:105B6C0010882034006802682243026081F3108898
:105B7C001FE08168B94202D1016900291ED0124A86
:105B8C000199009C19700267EFF3108185F310885E
:105B9C00026813682343136081F31088EFF31081BC
:105BAC0085F310882A07006883681343836081F3A8
:105BBC001088002002B0F0BD044ACAE7014ADFE7B2
:105BCC00FF010000E15B00087D5D000827B50008BF
:045BDC0071AF00089D
:105BE000F0B585B004460168C8690D688B68264623
:105BF0005C36B788F26A222A00D093E00393202112
:105C00000191B189002900D192E00199084000D1A9
:105C10008EE00121184608400390049108020540D7
:105C20000095029707E0204605F0A1F9009DB8060F
:105C3000029F00D47CE02068416A3940A26D118047
:105C40007188491E7180911CA165C769790732D09E
:105C50006A426A41FB07049B00D01346002B04D123
:105C600001220262336B13433363039B5A425A414E
:105C7000BB07049B00D51346002B05D1022202620C
:105C8000326B042313433363039B5A425A41002966
:105C9000049900D51146002905D104210162306B19
:105CA000022101433163306B002804D0204605F007
:105CB0005BF90020306370880028B8D1EFF31081C1
:105CC000012080F31088020223681D6895431D603F
:105CD00081F31088EFF3108180F3108822689368B5
:105CE000244D2B40936081F310880199F1620021CB
:105CF0002167E26E012A96D1E166EFF3108180F30D
:105D000010882268136810208343136081F3108881
:105D10002168CA69D20600D508623188204605F09C
:105D200024F983E78869082202438A6105B0F0BD3F
:105D300070880028FAD0B1898842F7D2EFF310803A
:105D4000012181F310880B4A521C23689D6815407D
:105D50009D6080F3108808482067EFF3108081F37E
:105D6000108821680A68019B1A430A6080F3108832
:0C5D700005B0F0BDFEFFFFEF27B50008F6
:105D7C00F0B585B004460168C8690D688B68264685
:105D8C005C36B788F26A222A00D095E00393202172
:105D9C000191B189002900D194E00199084000D10A
:105DAC0090E0012118460840039004910802054038
:105DBC000095029707E0204605F0D3F8009DB80641
:105DCC00029F00D47EE02068406A3840A16D0870C4
:105DDC007088401E7080A06D401CA0652068C7694B
:105DEC00790732D06A426A41FB07049B00D0134604
:105DFC00002B04D101220262336B13433363039BE8
:105E0C005A425A41BB07049B00D51346002B05D1BF
:105E1C0002220262326B042313433363039B5A4204
:105E2C005A410029049900D51146002905D10421B5
:105E3C000162306B022101433163306B002804D0C6
:105E4C00204605F08BF80020306370880028B6D10E
:105E5C00EFF31081012080F31088020223681D6883
:105E6C0095431D6081F31088EFF3108180F3108847
:105E7C0022689368244D2B40936081F3108801991C
:105E8C00F16200212167E26E012A94D1E166EFF301
:105E9C00108180F3108822681368102083431360EC
:105EAC0081F310882168CA69D20600D5086231884E
:105EBC00204605F054F881E78869082202438A617C
:105ECC0005B0F0BD70880028FAD0B1898842F7D2AD
:105EDC00EFF31080012181F310880B4A521C2368C8
:105EEC009D6815409D6080F3108808482067EFF38B
:105EFC00108081F3108821680A68019B1A430A609C
:105F0C0080F3108805B0F0BDFEFFFFEF71AF000805
:105F1C00F0B581B000283AD016460F4604460093DF
:105F2C00054680356868002803D12870204604F0A7
:105F3C00C3FB24206860206801680125A943016027
:105F4C002046FFF771FB012822D0A06A002802D05E
:105F5C00204604F023FF0120820321688B68134341
:105F6C008B60C2038B6893433B438B607205009B31
:105F7C001B0413430A68084D15401D430D600A6845
:105F8C0002430A602046FFF757FC054600E0012556
:0C5F9C00284601B0F0BDC046FFFF00FC2D
:105FA800F0B581B0054668352A7E012A02D1022063
:105FB80001B0F0BD2422EA6106683768326801241E
:105FC800A243326007225207B36893430B43B3607E
:105FD800406E0028204615D00097B768B068400F7B
:105FE8000D49095C0D4A105CC00004F0FFFB044633
:105FF8003801009F400F0849095C084A105CC0003E
:1060080004F0F4FB28806C8037600020287620217B
:10601800E96101B0F0BDC0467BBD000873BD000852
:10602800F0B581B0054668352A7E012A02D10220E2
:1060380001B0F0BD2422EA6106683768326801249D
:10604800A243326007225206B36893430B43B360FE
:10605800406E0028204615D00097B768B068400FFA
:106068000D49095C0D4A105CC00004F0BFFB0446F2
:106078003801009F400F0849095C084A105CC000BD
:1060880004F0B4FB28806C8037600020287620213B
:10609800E96101B0F0BDC0467BBD000873BD0008D2
:1060A800F0B5FFB0FFB095B0FFAD3C3508920E4695
:1060B80003905449694408600021534868440160CA
:1060C8000EA8E96028600124A0026860C843059012
:1060D80009940C9508E02B4600F02EFAA1E0099CE3
:1060E800E968002900D522E20D913178761C25292E
:1060F8000AD0002900D100E26A68AB68581C9042B7
:1061080028D99342ECD12EE0002730780246233A72
:106118000D2A15D80221C0467A44127952009744B4
:106128000B0F0F0F0F0F0F0F0D0F090F0F060F4358
:10613800761CEAE72146FAE70821F8E70421F6E7A2
:106148000921C94302463A3A00258A4216D22C460A
:10615800324620E02A68D154A860E968491CE96001
:106168006A689042BCD12968286904F07DFCA96856
:10617800884200D0D1E10020A860B1E700240A23BA
:106188005C432418303C721CDB43707806463A3E68
:106198009E421646F3D82E2814D1501C5278134626
:1061A8003A3B8B4201D206460CE000250A214D43BA
:1061B800AD18303D461CC943427810463A388842EB
:1061C8003046F3D83078FB210140761C6829F9D095
:1061D80001465839202931D87944097949008F4432
:1061E80022202020202020202020203A4620202065
:1061F8002020202020202020672020742015202007
:106208002200C0464804000040040000089A1068B4
:10621800011D1160016800940197FFA83C300A2213
:1062280059E70C9D5BE7089A1068011D1160016829
:1062380000940197FFA83C3010224CE72528F0D1A4
:106248000C9D6A68A968481C9042099C7CD99142B7
:1062580000D045E787E708990B68181D08600C9D72
:106268006A68A968481C90425FD9084665E0089AA0
:106278001068011D11600168C81706914140081A8D
:1062880001220A2809D30B920A210A9004F0AEFAD7
:106298000B9A521C0A996329F5D8AA4200D82A46B3
:1062A800002C0D994ED00698002851D4002050E0BB
:1062B800089A1068011D11600168002008230093E6
:1062C8000190FFA83C30102206E7089A1068011DCB
:1062D800116005680C998868CC6804E038466D1C24
:1062E8000D9100291DD4297800291AD0471C0C9B30
:1062F8005A68974204D907460D999742EED106E0AD
:106308001A681154641C5A6821469742E6D11968E4
:10631800186904F0A9FBB84200D0FBE00020214630
:10632800DDE70C9DA860EC60D9E61A682B685A5422
:10633800A860E968491CE9606A68099C904200D035
:10634800CEE610E700230AE02A682523535403E722
:1063580001200421394089080143631A0D9902205C
:1063680038400490099C0B9201D0002D3DD0F807CD
:106378003BD1002B39D00C9988680A90C9680791DD
:106388000D9806E00A9400280D9B099C0B9A00D5ED
:106398009DE0591E0D91994220D29A421ED20A9927
:1063A8004C1C0C9B5A68944203D90C469442E9D180
:1063B80009E00846196820220A540798401C5A68C0
:1063C80007909442DED11968186904F04DFBA04289
:1063D80000D0A4E000200A900798D4E702460C9960
:1063E8000A9888600798C860114600296DD40698F5
:1063F800002804D4780729D50D912B2103E00D91AD
:10640800404206902D210A930C9C6268A368581C90
:10641800904202D918460D9906E02268D154A0602E
:10642800E168491CE1606268099C90420BD10C9CB0
:106438002168206904F018FBA16888426DD100200A
:10644800A060E168099C00290A9B3ED404980028B2
:1064580048D001203840284344D1002B42D00A4676
:106468000C99486804908868C968079111460B9A86
:1064780005E0204600290A9B099C0B9A28D40D9018
:10648800581E0A90984228D29A4226D20B460D9856
:10649800441C0C994A68944204D90446194694420B
:1064A800E7D108E0096830220A540799491C079186
:1064B800049A9442DDD10C980168006904F0D4FA7A
:1064C800A0422CD100200799D4E70C9D08E60A9831
:1064D8000C9DA8600798E86002E60C9A0D989060F9
:1064E8000798D060069900930197FFA83C300A22CC
:1064F8002B4600F021F80C9DF2E50D99002916D0E5
:10650800AA68002A11D00EA9039804F0ADFAA86869
:10651800E9680BE00C988760C460059907E00C985F
:1065280084600799C160059901E0002009180846B0
:086538007FB07FB015B0F0BD8B
:10654000F0B585B001930290012403919142264653
:10655000049207D30846114604F04CF9049A761CBD
:106560009042F8D20B980A9A01998E4200D80E46B2
:106570000440002A009418D0002C16D1800701D4C2
:10658000202700E030270198002800D02027029C17
:10659000002A0AD0964208D220463946154604F011
:1065A00053FD6A1EE0680028F2D50298C0680028F2
:1065B00040D40124019F02E07F1E04994C43022F26
:1065C000FAD203982146154604F014F92A46049994
:1065D0008842F3D20196039E03963046214604F08A
:1065E00009F907461448C15D029E304604F02CFDAF
:1065F000F068039E002809D46743F61B2046049FD9
:10660000394604F0F7F8BC420446E5D20098002869
:10661000019E0FD0002D0DD06C1EAC420AD2AE42AE
:1066200008D22021029D284604F00EFDE8680028CB
:0C6630002546F1D505B0F0BD83BD000883
:10663C0070B584B03C213848002545542C210126E6
:10664C004654C56402218163466345628562062116
:10665C00C161867605830824304932030263021D2A
:10666C00157701607105B20742608560C5600161F4
:10667C004461039502950195FCF716FE002801D0A4
:10668C0002F0FEFA2648039002950196224801A9D1
:10669C00FDF746F8002801D002F0F2FA0395042029
:1066AC000290204801901C4801A9FDF739F80028F8
:1066BC0001D002F0E5FA02941B480190164801A99A
:1066CC00FDF72EF8002801D002F0DAFA0C20029027
:1066DC0016480190104801A9FDF722F8002801D0B6
:1066EC0002F0CEFA10200290114801900A4801A93C
:1066FC00FDF716F8002801D002F0C2FA142002901F
:10670C000C480190044801A9FDF70AF8002801D0B3
:10671C0002F0B6FA04B070BD8805002000240140D8
:10672C0004FFFF0702000004040000080800000C2E
:08673C008000001C4000001861
:10674400F0B595B0044600261496139603A8001DD0
:10675400302104F0D3F920682649884201D015B0CD
:10676400F0BD01940127B803039003A8FEF7E4FBEE
:10677400002801D002F088FA38051F49CA6802438C
:10678400CA60CA68024002920298086838430860E6
:106794000868384002901296CF2010900298032582
:1067A40011950524200710A9FDF7F2FE2803134DC7
:1067B40028622020B9023A028023114F2F606C60B6
:1067C400AE60EE602B616A61A961E8612846FDF75D
:1067D400FFFB002801D002F057FA0198A862056572
:1067E4000C2000210A46FDF79BFA0C20FDF7B8FAAD
:1067F40015B0F0BD0024014034100240A80F002061
:046804000800024046
:1068080080B50B4801210162002110220723836013
:10681800C26001614161816106490160FF21023165
:106828008180FDF7DFFA002801D002F02BFA80BD45
:0868380018120020003002409C
:1068400081B000680849884201D001B0704701203A
:10685000000306490A6802430A6009680140009182
:10686000009801B07047C046003002403810024026
:1068700010B58AB0134814490160002409940894A3
:106880000794069404F0C9FD002801D002F0FEF937
:10689000059404940394029401940A4801A90022E7
:1068A000FDF70CFB002801D002F0F0F9054801A922
:1068B0001022FDF703FB002801D002F0E7F90AB02F
:0C68C00010BDC046EC0500200074004034
:1068CC0070B586B00024059404940068144988427D
:1068DC0001D006B070BD01204107124A93680B43EA
:1068EC00936093680B400093009911680143116009
:1068FC00116801400091039403250295302001900A
:10690C0000980520000701A9FDF73EFE1120032188
:10691C000022FDF701FA1120FDF71EFA06B070BD3A
:08692C00007400403410024029
:10693400F0B581B016490868012210430860154873
:10694400002380244025144E03273F03076206607A
:106954004360D602570291038160C56004614761B8
:106964008661C3610A490968114000910099FDF7E5
:106974002FFB002801D002F087F909200121002211
:10698400FDF7CEF90920FDF7EBF901B0F0BDC046E3
:0C699400381002404C0F00201C00024094
:0869A00000487047EE070000FB
:1069A800F0B585B0FDF776FD002801D0012434E06C
:1069B800012046021A4D2968B14329600224019436
:1069C8000490184800680006400E801E039001A835
:1069D8006946FDF77FFD00281AD13720C443124FBE
:1069E800124DE1192819826BC36B0120FDF7D8FC01
:1069F80000280BD10834F4D10949086830430860ED
:106A0800FDF75CFD411E8841840006E00324044D27
:106A1800286830432860FDF751FD204605B0F0BDD9
:106A280000200240E075FF1F38F0010838050020FB
:106A3800F0B583B03721CB4302461632264C27499E
:106A48001D5DCE183827F5555B1CF9D30B681380EC
:106A58001B0C53808B8A02934B8A01938B8900937A
:106A68004E890F89CC888B88CD8A958543830B8B7B
:106A7800D38584834B8B1386C7838B8B5386CB8BB1
:106A88009386CB89D3860B8A13870685009B438719
:106A9800019B8387029BC3870B8C114C2380002B9F
:106AA80001D0012353870A6B0281120C4281888D21
:106AB800382805D1C88D002805D0032003B0F0BDC3
:106AC800022003B0F0BD2420085C6538411E8841CF
:106AD800800003B0F0BDC04638F00108380500203A
:046AE800120E00206A
:106AEC00B0B5C38A048B058D1B4A5581458B9580A7
:106AFC00858BD580C58B1581458F9581858F55826A
:106B0C00C58F95822404E3181360034616339C8DBD
:106B1C00D482DC8D14831C8E54835C8E94839C8E67
:106B2C00D4835624045B1484DC8ED4811B8F2424E0
:106B3C006525155513823823D362936A5B1C9362C7
:106B4C00002904D001894089000440181063FFF724
:0C6B5C0025FF411E8841B0BD3805002017
:106B6800B0B50B490B48024638C938C238C938C2D3
:106B780038C938C22421652242543821C162816A49
:106B8800491C8162FFF70CFF411E88414000B0BDDF
:086B980024AB000838050020C1
:106BA000024800786538411E8841704724F001088A
:106BB000F0B585B0FDF772FC002801D0012434E067
:106BC000012046021A4D2968B1432960022401942C
:106BD0000490184800680006400E401E039001A86B
:106BE0006946FDF77BFC00281AD11720C443124FD9
:106BF000124DE11928198269C3690120FDF7D4FB00
:106C000000280BD10834F4D10949086830430860E2
:106C1000FDF758FC411E8841840006E00324044D22
:106C2000286830432860FDF74DFC204605B0F0BDD4
:106C300000200240E075FF1F18F8010870050020D1
:106C400080B5064800210182016041608160C16019
:106C5000FFF7AEFF411E8841400080BD7005002057
:106C600030B50121090240181721CA430D4B0E49C6
:106C7000D45C8D182C76521CFAD30A8802804A887C
:106C800042808A888280CA8802820A89C2804A89B0
:106C900002818A894281CA898281098AC181002050
:0C6CA00030BDC04618F801087005002047
:106CAC0080B501210902425A41180C4802804A88D9
:106CBC0042808A8882800A8AC280CA8802810A89B4
:106CCC0042814A8982818A89C281C9890182FFF7FE
:106CDC0069FF411E8841400080BDC0467005002000
:106CEC00F0B587B00024069449480168042211438A
:106CFC000160016811400191019901682022114342
:106D0C000160016811400191019901680125294335
:106D1C000160016829400191019901680222114327
:106D2C000160016811400191019901680822114329
:106D3C00016000681040019001986903354E30469F
:106D4C002A4604F078FBA9033046224604F073FB74
:106D5C0031481F273946224604F06DFB2F4829463F
:106D6C00224604F068FB0594049403950320400329
:106D7C00029002AE27483146FDF706FC04940394BA
:106D8C00E8030090029023483146FDF7FDFB059483
:106D9C00049403950297204F38463146FDF7F4FBD7
:106DAC0004950394FF200002029038463146FDF70B
:106DBC00EBFB0494039409200002029005200707C2
:106DCC0038463146FDF7E0FB04950394C020029051
:106DDC0010483146FDF7D8FB0495039400980290B7
:106DEC0038463146FDF7D0FB059404940395029583
:106DFC000A4F38463146FDF7C7FB049503940C2027
:106E0C00029038463146FDF7BFFB07B0F0BDC046D7
:106E1C00341002400008005000040050000C0050D8
:106E2C0070B50D4606460A49002003F035FE0020D9
:106E3C00314603F031FE0749002003F02DFE0020FF
:106E4C00294603F029FE0449002003F025FE70BDFD
:0C6E5C0093BD000899AB000885B8000841
:106E680070B50D4606460A49002003F017FE0020BB
:106E7800314603F013FE0749002003F00FFE0020FF
:106E8800294603F00BFE0449002003F007FE70BDFD
:0C6E98009BBD000899AB000885B80008FD
:106EA40070B50D4606460A49002003F0F9FD00209E
:106EB400314603F0F5FD0749002003F0F1FD002001
:106EC400294603F0EDFD0449002003F0E9FD70BDFF
:0C6ED400A3BD000899AB000885B80008B9
:106EE00000B589B0D74801260660FCF769F900F0C3
:106EF000A9FCFFF7FBFEFFF71DFDFFF79FFB03F06B
:106F0000A7FBFFF781FCFFF7B3FC03F0CFFA03F018
:106F1000B1FA03F061FA03F039FA03F011FA03F061
:106F2000DFF903F073FAC84C204608308721490086
:106F300003F0E6FD0020C54921606060C448FEF70B
:106F400061F9002803D0C348C349FFF7ABFF002015
:106F5000C24904F038FBBF48C149FFF767FFC14D84
:106F60002868C1490140C148081811280FD8C049F4
:106F70007844007940008744080A0A0A0A0A0A0A83
:106F80000A0A0C0A0A0A0A0A0E0FBA4904E0BA49A8
:106F900002E0BA4900E0BA49AE4C2046FFF746FF8E
:106FA0002868030C0027B7493846224604F00BFB3B
:106FB00004F06BF80246B449384604F004FBFFF7CE
:106FC000EFFC0246B149384604F0FDFAB04996227A
:106FD000384604F0F8FAFDF739FF0246AD49384665
:106FE00004F0F1FAFDF732FFAB4988420AD8994C18
:106FF000AA492046FFF756FFA9492046FFF752FF4E
:10700000FCF7CCFE00F05EFC00F08AFCFFF7C8FD48
:10701000002807D08F48A349FFF726FFFFF7A4FDFC
:10702000FFF70EFE8848FFF707FD002803D08948C8
:107030009D49FFF737FF844C2046FFF711FE0028DB
:1070400003D084489949FFF72DFF3002215A491C8B
:107050002152E18F6E204843642103F0CBFB402195
:107060006052934806604620205A4A21615A4143A3
:1070700090480160E08B9049022204F009F8E08A10
:10708000218B628B8D4B01938D4B00936F2A00D027
:107090000226652A00D0374609040918894D8A4B13
:1070A00028463A4604F04AF8884804F052F9002885
:1070B00001D0874906E08548FCF7E6FD002800D1AD
:1070C00046E384496348FFF7EDFE834800263146D6
:1070D00003F028FE074610217F4803F023FE0790A7
:1070E0007E495C4A30463B4604F06DFA7C4908967E
:1070F0000020584A079B04F066FA0120069000F031
:1071000047FC724877490622FCF7BAFA002803D0F8
:1071100050487549FFF7C6FE744801680422914340
:1071200001606D48314603F0BFFD10216A4803F04D
:10713000BBFD694831463246334603F0DEFD664802
:1071400010213246334603F0D8FD00F0A7FC684911
:107150006848086068486949016069480160694891
:1071600001606948016069480160694869490160D6
:1071700006980102049141020391C043079008E080
:107180000020208400F0A6FFFCF760F8B04200D099
:10719000FDE000F01BFF284604F023FA002810D081
:1071A000284602F0CBFD022807D15B480068002882
:1071B00007D0284602F012FE03E088202221424A2E
:1071C00011505427E05B55490988401A414241411A
:1071D00052202152394801801A4800680028CFD037
:1071E0002621208C0028CDD0695C0029CAD14C49C9
:1071F000884200DDA2E0411E1D2900D91EE249009F
:107200007944898849008F44900039014A011D0260
:1072100069011D021D021D021D0280011D021D02C9
:107220001D021D021D021D021D021D021D02830101
:107230001D021D021D021D021D021D021D021D0256
:107240001D028D00F4120020FC0C0020CA00010079
:107250009C10002045BB00084ABB00085FBB00082B
:1072600064BB000800580140FF0F0000AAFBFFFFAD
:1072700087B80008CBB80008ADAB0008A9B8000873
:10728000EDB80008ABBD00080FB90008C7BD000885
:1072900045B9000875BB0008FF8FD003FBBD00088F
:1072A000FEB5000813BE000886BB000811B6000832
:1072B000C01200206C04002000040050B61300200F
:1072C000AC040020C00A0020BC0E0020880500206D
:1072D000D4BB000840B60008EC050020E5BB000860
:1072E00012BC0008D213002067B900080800024051
:1072F00044130020157F000840130020F9010020EE
:107300003C1300207C1300206C1300208C13002001
:1073100048130020657F000874040020120E00202E
:107320004F4F000002F0D4F92AE700212046FFF772
:10733000DDFB002800D111E1FB490CE1FB4988424B
:107340000FDCFB49884200D1E6E0FA49884200D1CF
:10735000E6E0F949884200D074E1F848F849016054
:107360000EE7F849884200D1E4E0F749884200D1AD
:10737000EAE0F649884200D064E1FC480068FC4934
:10738000884200D0FCE6F948FA490160F8E6074671
:10739000F64800688047F84800688047FB48006866
:1073A0008047F64800688047F94800688047F948F8
:1073B00000688047F24E30684000306005200007CA
:1073C0000121890303F0B7FC31680143316002D029
:1073D000384600F0B9FE384601F044F8384601F06E
:1073E000E5FA0898381AE74988420ED3EB48E6498F
:1073F000FFF71CFDEC4800680028089705D02046E0
:10740000FFF754FC0020E8490860A08D022800D155
:10741000AFE001283E4600D0BBE6FB4800680128EB
:1074200000D026E10798FF38E34909684A6802401E
:107430004A604868E84A1040486004980860039829
:107440000860F84E3046FDF74BFF326830460026A4
:10745000566207991161FDF70BFF09200590FCF7B3
:107460008DFCEA202652F048F04901600598FCF7AF
:1074700079FCD648EE4901603E468AE6608B6F286B
:1074800000D1C3E0652800D0CAE0E08A218BC84A59
:107490000092C64A0192090409180022C9E0FFF7C8
:1074A00063FB0028BD4F03D03846D249FFF7FAFCF2
:1074B000FFF7C6FB2046FFF7BFFA002803D0384687
:1074C000B749FFF7EFFC2046FFF7CAFB002800D1C1
:1074D00056E6B248B349FFF7E5FC51E6AF48C64966
:1074E000FFF7A4FCE15BBD480088814208D1002180
:1074F0002046FFF7FBFA5620205AE053B749088090
:10750000411E8841502160523AE602F029F937E6DF
:10751000002000F03DFA33E6AB48AE4908602FE6A4
:10752000AB480068A849884200D029E6A848AC4981
:10753000016025E6A6480068A349884200D01FE6FE
:10754000A348A84901601BE601212046FFF7CEFAB7
:10755000002803D0A6499148FFF7A4FC2046FFF776
:107560006BFA002800D10BE68C488D49FFF79AFC96
:1075700006E6B0480068411E48424841A2490968F1
:107580000129069900D0014601297FD1AA48007837
:1075900000283E4600D0FCE50798FF388649096878
:1075A0004A6802404A6048688B4A10404860049824
:1075B0000860039808609B4E3046FDF791FE3268E4
:1075C00030460026566207991161FDF751FE0920E9
:1075D0000590FCF7D3FBEA202652934893490160BB
:1075E0000598FCF7BFFB88480068012802D177485E
:1075F0008F4901608F480068012802D17348904983
:10760000016006988C4908703E46C2E5E08A218BED
:10761000674A0092654A019209040918012208E0AC
:10762000E08A218B624A0092604A0192090409189B
:10763000022228465F4B03F081FDA1E57D218900F0
:10764000884260D06D48026807991161002757622F
:10765000FDF70EFE0028514904D008466849FFF79F
:1076600021FC4E494C48076008466649FFF7FCFB81
:1076700086E566480068012815D06548006801283D
:1076800022D06448006801282FD082E55F48006856
:1076900001280CD16848007800283E4600D078E5E3
:1076A00006986549087049485D49016071E5584888
:1076B000006801280CD16048007800283E4600D0C0
:1076C00067E506985C49087040485449016060E5E8
:1076D0005048006801280CD15748007800283E46E1
:1076E00000D056E506985449087038484A49016068
:1076F0004FE5514E31785148026838469047002096
:1077000030703E4645E52F480068002181604161A8
:10771000EA202152BFF34F8F334834490160BFF351
:107720004F8F00BFFDE7C04615BB00086D9D0000F0
:10773000504F0000F9750000C57600004813002086
:10774000657F00086E9D0000E3C4000058EC000057
:10775000194803F05CFE3F210143009100201749C6
:10776000174A0E4B03F02FFFAFE4C0468C130020E6
:10777000F9010020ED970008401300203C13002081
:1077800060040020C1D401003FBC00084413002065
:107790007C1300206C130020F412002045BB00086D
:1077A00086BB000811B60008C0120020B6130020E6
:1077B000AC040020BC0E002088050020B3BB0008EC
:1077C0003FBE0008EC050020F90100206C130020EA
:1077D0008C13002048130020FFFDFFFF120E002035
:1077E00071980008659900080CED00E00400FA05A6
:1077F0009BBF000852B800083BB80008E810002002
:10780000BFBF000855BD0008BC120020D4120020E4
:10781000D8120020D0120020A58B0008398B000858
:10782000D18A0008801100202C13002001000020C4
:107830006D8A0008E0120020B41300209C13002081
:04784000198C000897
:1078440070B592B00025069501267002FCF7F8FF8A
:10785400700711907006109070040F9010200E9015
:107864000D9502240B940A9640200990300207904B
:10787400300405900B20049003200C90C002089063
:1078840004A8FDF707F8002803D00B480B49FFF7BD
:1078940007FB039502950720009001946846022196
:1078A400FDF718FA002803D003480449FFF7F8FA53
:1078B400FDF722FB12B070BD45BB000830B80008CC
:1078C400F0B581B0144C20460121012203F0B7FD2C
:1078D400022100912046012203F0B1FD042120463B
:1078E400012203F0ACFD7D26F000FBF7B3FC0A484F
:1078F4000121002203F0A3FD074D28460099002230
:1079040003F09DFD28460421002203F098FDB000F9
:0C791400FBF7A0FC01B0F0BD0004005027
:10792000B0B5134D29681348134C30232246FCF799
:10793000C7FB002804D011481149FFF7B3FAFEE74E
:107940000E481049FFF772FA7D20C2000948002155
:10795000FCF79CFC002804D008480B49FFF7A2FA6A
:10796000FEE706480949FFF761FA2C60B0BDC04642
:1079700008ED00E04C0F00200006002045BB000889
:1079800085B9000857B60008C3B9000847BE00080B
:10799000F0B581B00546FBF759FC04462D4E012792
:1079A0003A02002D07D13068201A1146F43188427E
:1079B00001D801B0F0BD00922748FDF791FC27499E
:1079C000888D002800D0346000268E85FD4328462F
:1079D000FF38234909684A6802404A6078024A68C9
:1079E00082434A60009A0A6008601E4C2046FDF7F8
:1079F00077FC2068466205612046FDF739FC0920C6
:107A0000FCF7BCF9EA20154F3E52174817490160B0
:107A10000920FCF7A7F9164801680D61154A164BB5
:107A20001360164A164B1360164A174B13604E62CA
:107A3000FDF71EFC452080003E52892040003E524A
:107A40001248066012480660124806601248066036
:107A500001B0F0BDE412002034110020FC0C002025
:107A600088050020801100202C1300200100002038
:107A7000CC1100206C1300204D8D00087C130020D9
:107A8000C58D000840130020518E0008D41200203C
:0C7A9000BC120020D8120020D0120020F0
:107A9C00F0B583B001252E02F54C2046314603F09B
:107AAC0044F902956D02012825D12046294603F0A0
:107ABC003CF901281FD10127B902204603F035F902
:107ACC00012818D13D46F902204603F02EF9002872
:107ADC0000D1FEE0E748E549FFF7A2F9E748F54990
:107AEC00FC4AFD4BEA4FFD4E3E60036042608160F4
:107AFC00C160002070E12046314603F016F90028E1
:107B0C0025D12046294603F010F901281FD1012761
:107B1C00B902204603F009F9012818D1F9022046D0
:107B2C0003F003F9002800D1FCE0D248EF49FFF73D
:107B3C0077F9D248DF49E04AE04BD54DE04E2E6054
:107B4C003D46036042608160C160384644E1204696
:107B5C00314603F0EAF8012824D12046294603F0E7
:107B6C00E4F800281ED10127B902204603F0DDF805
:107B7C00012817D1F902204603F0D7F8002800D1CC
:107B8C00E2E0BC48D249FFF74BF9BC48C949D14A9D
:107B9C00D14BBF4DD14E2E60036042608160C160FD
:107BAC00022018E12046314603F0BFF8002824D10A
:107BBC002046294603F0B9F800281ED10127B90246
:107BCC00204603F0B2F8012817D1F902204603F041
:107BDC00ACF8002800D1DCE0A648B549FFF720F945
:107BEC00A648B449B44AB54BA94DB54E2E600360B6
:107BFC0042608160C1600320EDE02046314603F015
:107C0C0094F80299CF0201280CD12046294603F0A2
:107C1C008CF8012806D101908102204603F085F8EA
:107C2C0000283DD02046314603F07FF800280BD1C8
:107C3C002046294603F079F8012805D18102204617
:107C4C0003F073F8002855D02046394603F06DF840
:107C5C00002811D087488849FFF7E2F887488849FF
:107C6C00884A894B894D056043608260C1608848B1
:107C7C0088490160042010E07E488749FFF7D0F85E
:107C8C007E487F497F4A804B804D0560436082600F
:107C9C00C1607F48814901600C2002990D469CE02F
:107CAC00019E2046394603F040F800285DD071480B
:107CBC007D49FFF7B5F871487149724A724B734DA3
:107CCC00056043608260C1607148724901600420A4
:107CDC005CE068488749FFF7A3F868487549814A12
:107CEC007D4B6B4F804E3E60036042608160C16093
:107CFC00082071E02046394603F017F8002859D0C7
:107D0C005C486749FFF78CF85C485D495D4A5E4BFF
:107D1C005E4D056043608260C1605D485D490160F5
:107D2C00052058E053487249FFF77AF853486149E7
:107D3C00654A624B564D654E2E6003604260816011
:107D4C00C1600920012547E04A486549FFF768F8FA
:107D5C004A485849634A604B4D4D634E2E60036050
:107D6C0042608160C1600A2035E042484F49FFF70C
:107D7C0057F842484249434A434B444D05604360DF
:107D8C008260C1604248454901600C200299354629
:107D9C0023E038484B49FFF743F8384845494A4AED
:107DAC00464B3B4D494E2E60036042608160C16082
:107DBC000B2010E02F483B49FFF732F82F48304991
:107DCC00304A314B314D056043608260C1603048B0
:107DDC00324901600D2000250299474F78854748AC
:107DEC0005700903204602F0A0FF002803D0444888
:107DFC000021016006E0424801210160788D1021CC
:107E0C0001437985012675032046294602F08DFF32
:107E1C00002803D03B480021016005E0394806608A
:107E2C00788D20210143798531022046FCF780FCB6
:107E3C0071022046FCF77CFCB1022046FCF778FC72
:107E4C00F1022046FCF774FC31032046FCF770FC71
:107E5C0020462946FCF76CFCB1032046FCF768FC75
:107E6C00F1032046FCF764FC03B0F0BD8AB60008B1
:107E7C000004005045BB000874BC000878120020B8
:107E8C0061950008E9940008759400080D940008A9
:107E9C009C1300200596000877BE0008719300081B
:107EAC0061B70008CBBA000836B70008A1BA0008C1
:107EBC000BB70008F9010020D1920008819100084D
:107ECC004D92000877BA0008C19100080191000892
:107EDC00E0B6000861900008118F0008DD8F0008E3
:107EEC004DBA0008518F0008918E0008B5B60008F5
:107EFC0023BA0008F9B90008FC0C0020FB01002093
:087F0C00DC1200200413002028
:107F1400F0B581B0FBF798F904460D4F3868201A84
:107F24000C490E78002E03D033280ED3002203E030
:107F34000949884209D9012208480125294603F044
:107F44007EFA3C606E400348067001B0F0BDC04646
:107F540094130020CC130020B6030000000400504A
:107F640080B511480068002181604161EA220F4810
:107F740081520F490F4A0A600F490968002900D04D
:107F840080BD0E490A68002A07D111221201835AC2
:107F94005B1C83520A480122026001200860FBF73F
:107FA40053F90849086080BDEC050020FC0C002052
:107FB4002C130020F9010020D4120020D01200203C
:087FC400C0120020640400203B
:107FCC00F0B581B0FBF73CF9314908600A683148DB
:107FDC000368D21A022A2ED3096801602E4D688FCD
:107FEC002E4909684018E821685201B24B208000E4
:107FFC0048432B4902F0D8FBD8216B5E294A146800
:10800C00E31AC318963BD817800C181880136852C3
:10801C001360EA26AB5B002B0AD0234C2778002F89
:10802C000BD0022B10D100042649884212DD02E04D
:10803C001D480021017001B0F0BD00206852106095
:10804C000120207001B0F0BD032BF4D100041849BD
:10805C008842F0DB154F38680028ECD10920FBF77B
:10806C0087FE14480068002181604161A9531248C1
:10807C00124901600920FBF76FFE87204000295A46
:10808C00491C2952012038600D49086001B0F0BD2F
:10809C00AC130020B0130020FC0C0020C4120020F4
:1080AC00FF0F0000A8130020D0130020D8120020CE
:1080BC0001003C00EC0500202C130020F9010020ED
:0880CC00C0120020FFFFC3FFFA
:1080D40080B5FBF7B9F816490A68904200D180BD13
:1080E400086002F09FF8082002F0DAF8002806D0B1
:1080F40010481149FEF798FE01F0E8FA80BD082007
:1081040002F0DCF8002806D00A480C49FEF78CFE81
:1081140001F024FB80BD042002F0C2F80028DED068
:1081240004480749FEF780FE0020FFF72FFC80BDBE
:108134003813002045BB0008F5BA00088CB70008C6
:04814400C3BE0008AE
:10814800F0B581B0A0490A68821A4E2A00D238E1F7
:10815800086000259D499E4C9E4B2846224603F008
:108168002EFA9D4F9D4A28463946234603F027FAA2
:10817800D8209B4E325E9B49284603F020FA2846B9
:108188003946964A234603F01AFAFC20325E96498D
:10819800284603F014FA28463946904A234603F045
:1081A8000EFAEC20325E9149284603F008FA284678
:1081B80039468A4A234603F002FACC20325A8C49BF
:1081C800284603F0FCF928463946844A234603F03A
:1081D800F6F9D220325A8749284603F0F0F92846A2
:1081E80039467E4A234603F0EAF9CA20305A824EBD
:1081F800824C0028324600D022468149284603F0A6
:10820800DEF928467449754A714B03F0D8F9C8203D
:108218007349085A002800D026467A490020324679
:1082280003F0CDF900206C4F39466C4E3246684B4E
:108238001C4603F0C4F974480068C26A73490020F8
:1082480003F0BDF9002039463246234603F0B7F95A
:108258006D480068026B6E49002003F0B0F90020F9
:1082680039463246234603F0AAF9EA205C49085AFF
:10827800002803D0012803D1674A06E0654A04E0D4
:10828800022801D0664A00E0644A00246549204675
:1082980003F095F9504D514A4D4F204629463B462B
:1082A80003F08DF9E2204E4E305E5F494143CA0F1C
:1082B80089148A180921C94351430818C11748402D
:1082C800431A5A49204603F07AF900202946434ABE
:1082D8003B4603F074F9F625705BC00704D0002014
:1082E8005349544A03F06BF95149534A204603F065
:1082F80066F93949394A364B002003F060F9705B5A
:10830800800704D500204A494A4A03F058F94849E9
:108318004A4A204603F053F92F49304A2C4B002093
:1083280003F04DF9705B400704D500204049414AED
:1083380003F045F93E49424A204603F040F92649F0
:10834800264A234B002003F03AF9705B000704D556
:1083580000203749374A03F032F93549394A20466F
:1083680003F02DF91C491D4A194B002003F027F989
:10837800705B800604D500202D492E4A03F01FF9B2
:108388002B49274A204603F01AF91349134A104B80
:10839800002003F014F92C48012102F0C8FC012840
:1083A80006D1002022492A4A03F009F9294A00E0A7
:1083B800264A1F49002003F002F92749002003F04C
:1083C800FEF801B0F0BDC04688130020C1BC00080B
:1083D8003FBE000845BB0008E3BE0008DBBE00083E
:1083E800FC0C0020EBBE0008F7BE0008C6BC000865
:1083F800A7B70008B2B700080BBB000803BF000806
:10840800CFBC0008D8BC0008EC050020BDB70008A8
:10841800C8B70008D3B70008D6B70008D9B700080E
:10842800DCB700080DBB000867660000E1BC000867
:10843800DFB7000813BF0008E2B70008E5B7000877
:10844800E8B70008EBB70008000C00502BBF000885
:0C8458001BBF000823BF000813BB000876
:10846400F0B589B0BD4909780029BD4D01D129462F
:1084740000E08721BB4C2268821A8A4200D81EE29F
:10848400CC26B94B995BB94A1268571AF9178F432E
:10849400B749CA886A43110B0A2251437918CF0895
:1084A4009F5301260296AD4D2E702060AF480160A7
:1084B400B8B21E46D021595A814203D2D033A84DB6
:1084C400AB4F06E0CE21715A8142A54DA84F01D988
:1084D400CE331880D220315AA64B1C68611ACC17AF
:1084E400A1437C886C43240B624389184A093252A5
:1084F400196090B2FC49884212D8FC4A11680029DC
:1085040019D1F621735A08241C437452832149005B
:10851400735A5B1C7352029B1360FA490B600AE0A6
:10852400F649884207D3F621725A08239A437252B5
:10853400F34900220A60D621715A814202D232469E
:10854400D63205E0D421715A814202D93246D4325E
:1085540010803888EC494143EC480818EC4902F093
:1085640027F9E221725EEB4B1C68A21A1018EA4A42
:108574008218D017C00E1018401170521A6004B23D
:10858400E621715E8C4202DD3146E63105E0E421EC
:10859400715E8C4202DA3146E4310880318D8C42BE
:1085A40013DA4B204843642102F022F9A0421DDD76
:1085B400DB480068002819D0F620315A029A91430A
:1085C4003152D6480021016010E0D44801680029E6
:1085D4000CD1F621725A029B1A437252812149002E
:1085E400725A521C72520360C6480360CD48006838
:1085F400401E414241414900F620325A26239A4303
:108604005118C94A1268521E534253419A005118D4
:10861400C64A1268521E534253415A0189183152B4
:10862400D823F05E0028009305D4DC21725A9042CE
:108634000ADCDA2105E0E021725A4042904203DC70
:10864400DE21725A904200DA7052B9490868F82261
:10865400B052B8480268FA23F252B74A1268B74BCC
:108664001B689A1A09688D18E917090F69180A1105
:108674004C21715A9142019201DC561A00E0002605
:10868400AF490968AF4A1268511A00684718F817C9
:10869400000F381804114E209649085A001B00DCBC
:1086A400361893487043A84902F082F8FC21914A95
:1086B4005052A2480560A348076017469E48019996
:1086C40001609F4804605F2084006643D18F304678
:1086D40002F06EF8EC217852EA257A5B9B48016837
:1086E400002A019404D19A4B994201D0984A09E096
:1086F400012A04D1974A914201D0964A02E0964A4F
:10870400914200D00260954C4021204602F011FBBA
:1087140006468021204602F00CFB914909784A4222
:108724004A41B11A4B1E9941CA23F952801A411E7B
:108734008841C8217852785B401E02281CD80098D2
:10874400385E032800DABCE0864801210A4602F0BC
:1087540076FE019978318448016012E0C01300204C
:10876400B80B000060130020FC0C002090130020C4
:10877400D2130020900400207A480121002202F044
:108784005EFE029E44203D5A784C2188A94214D0B2
:10879400B98F8D4211D956494A1E954201D9395291
:1087A4000D466948684302F023F846217852258033
:1087B4004A21795A41436E48016048203D5A6D4C24
:1087C4002188A94210D01E2D01D81F253D526A4888
:1087D40068436A4902F00CF84A2178522580462100
:1087E400795A41436248016005200007310202F0D2
:1087F400A0FA401E41424141FE2039524225785B95
:1088040000265F4CA15F814259D05E4802F002FA13
:10881400785BBA8F9042014600D811469042344AA0
:1088240001D3914204D9914200D3114679530846A9
:1088340020800196089644494843114601F0D8FF28
:108844000790514805900320860504964F480390ED
:10885400029806904B4803A9FBF792F8002803D02E
:108864004B484C49FEF71CFB03AC029820734A4862
:10887400059004964948039001980890795B324822
:1088840048431B4901F0B4FF07903E482146FBF7DB
:1088940077F8002803D03E483E49FEF701FB3948EB
:1088A40015490622FAF7EAFE002803D038483C4965
:1088B400FEF7F6FA3B48016804229143016009B0CF
:1088C400F0BD0028029E00DD5CE727490868012806
:1088D40001DB401E0860002800D053E72148012135
:1088E400002202F0ACFD4DE71F4E0000E012002014
:1088F400B80B0000FC0C0020D2130020C15D000066
:10890400E0120020C0120020140500000CE3F7FF61
:10891400EF06000054130020D4FEFFFFBC12002019
:1089240004130020D4120020D0120020D8120020FA
:10893400C8120020CC1200204C1300205813002031
:10894400501300205C130020FF0F00004013002090
:10895400518E0008718E0008058E00080008005032
:10896400FB010020000C005064130020BE13002003
:108974006C040020C213002000E2040040420F00F7
:10898400BA1300208805002004000008FFFF170028
:1089940045BB000830B8000840000018FFFF27005E
:0889A40067B900080800024059
:1089AC00B0B517490A68821A1A2A0FD30860154DF8
:1089BC00287840002870052000070124E10302F00C
:1089CC00B4F92978002802D0002911D0B0BD214378
:1089DC0029700D4801780029F8D104700B48016802
:1089EC00002908D00021016009480A490160B0BD86
:1089FC0005480170B0BD0460054807490160B0BD71
:108A0C001813002037050020B81300207404002030
:0C8A1C0044130020A18C0008157F000806
:108A2800B0B50D48006841680C4D294041600121EE
:108A38004A02436893434360090201600260084C9C
:108A48002046FCF749FC206800214162FF3505619A
:108A58002046FCF709FCB0BD88050020FFFEFFFF9B
:048A68008011002059
:108A6C00F0B587B005AD0F48288006AEC820308021
:108A7C00082003900C4F0297019500960B480C4967
:108A8C000C4A012302F01BFB022000960195029771
:108A9C000390094809490A4A012302F010FB07B068
:108AAC00F0BDC046C409000000040050781300203B
:108ABC0074130020701300201413002010130020D6
:048ACC000C13002067
:108AD000F0B587B005ADC820288006AE3080708024
:108AE0000D486880082003900C4F0297019500966E
:108AF0000B480C490C4A0224234602F0E6FA009681
:108B0000019502970394094809490A4A022302F091
:108B1000DCFA07B0F0BDC046C409000000040050F4
:108B20007813002074130020701300201413002009
:088B3000101300200C130020BB
:108B3800F0B589B005ADC820288007AE30807080B8
:108B48006880B0800D48A880082003900C4F0297D9
:108B5800019500960B480C490C4A032302F0B1FA20
:108B680002200096019502970390094809490A4A8C
:108B7800032302F0A6FA09B0F0BDC046C4090000FC
:108B88000004005078130020741300207013002094
:0C8B980014130020101300200C13002008
:108BA400F0B589B0002005AAC821115207AA1152B4
:108BB400801C0628F7D105AD0E48E88007AEF18089
:108BC400082003900C4F0297019500960B480C491E
:108BD4000C4A042302F077FA0220009601950297CA
:108BE4000390094809490A4A042302F06CFA09B0BF
:108BF400F0BDC046C40900000004005078130020F2
:108C0400741300207013002014130020101300208C
:048C14000C1300201D
:108C1800F0B58BB0002005AAC821115208AA11523C
:108C2800801C0828F7D105AD0E48288108AE31818F
:108C3800082003900C4F0297019500960B480C49A9
:108C48000C4A052302F03DFA02200096019502978E
:108C58000390094809490A4A052302F032FA0BB081
:108C6800F0BDC046C409000000040050781300207D
:108C78007413002070130020141300201013002018
:048C88000C130020A9
:108C8C0080B502480249FEF707F980BD45BB0008D4
:048C9C0030B80008E4
:108CA00080B5044801210A4602F0CBFB0248034983
:108CB000016080BD0004005044130020F901002031
:108CC00003480068002181604161024801807047CB
:088CD000EC050020E60D002078
:108CD800F0B589B005ADC820288007AE3080708017
:108CE8001048E8807D2080006880A880C830B08067
:108CF800F080082003900C4F0297019500960B48CE
:108D08000B490C4A042302F0DCF902200096019575
:108D18000297039008480949094A042302F0D1F947
:108D280009B0F0BDC4090000000400507813002009
:108D38007413002070130020141300201013002057
:048D48000C130020E8
:108D4C00B0B5074C08210022204602F074FB02212A
:108D5C002046002202F06FFB024803490160B0BDBF
:0C8D6C00000400506C130020F9010020EE
:108D7800F0B581B0FAF766FA04460D4E3068201A4D
:108D88000C4D2F78002F03D0C9280ED3002204E001
:108D980019214901884208D901220748102102F007
:108DA8004CFB3460012047402F7001B0F0BDC04635
:0C8DB80080130020C813002000040050AD
:108DC40080B504481021002202F039FB024803490F
:108DD400016080BD000400507C130020F9010020D4
:108DE40080B504481021012202F029FB02480349FE
:108DF400016080BD000400507C130020F9010020B4
:108E0400F0B581B0FAF720FA04460C4E3068201A07
:108E14000B4D2F78002F03D033280DD3002203E00D
:108E24000849884208D901220748042102F007FBB7
:108E34003460012047402F7001B0F0BD681300205A
:0C8E4400C4130020B6030000000400501E
:108E500080B504480421002202F0F3FA02480349D5
:108E6000016080BD0004005040130020F901002083
:108E700080B504480421012202F0E3FA02480349C4
:108E8000016080BD0004005040130020F901002063
:108E9000B0B5002901D0022523E013490A68821ADF
:108EA000124C23689A421ED908601148802101F0B3
:108EB00042FF454245410F490978002900D0054647
:108EC0000D480068A84202D10C490D4803E0A800F3
:108ED0000C4908580C49AA000C4B9850895821603D
:108EE000804705480560B0BDA4130020A8040020F9
:108EF00000080050FB010020A404002050AB000833
:108F0000F90100207812002048AB0008B0120020C0
:108F100010B50920FAF732FF074801F093F80B4823
:108F2000012101800548064901600920FAF71AFF6E
:108F300004480549016010BD650000202C13002085
:108F4000410300207C130020798D0008E60D0020ED
:108F5000F0B581B0184800684168184E3140416052
:108F60000125690242688A4342602A020260016068
:108F7000134C2046FCF7B4F9206800274762FF36FF
:108F800006612046FCF774F90920FAF7F7FEEA209B
:108F90000C4E37520C480D4901600920FAF7E2FEE9
:108FA0002120C000315A491C315209480949016049
:108FB0000948056001B0F0BD88050020FFFEFFFFF5
:108FC00080110020FC0C00202C13002089000020C0
:0C8FD0007C130020798D0008C0120020E6
:108FDC00B0B5002902D00020C54323E013490A682C
:108FEC00821A134C23689A421ED9086011488021BA
:108FFC0001F09BFE454245410F490978002900D0FC
:10900C0005460E480068A84204DAA8000E49085824
:10901C000E4901E00A490B48AA000D4B985089589B
:10902C002160804705480560B0BDC0463413002060
:10903C008C04002000080050FB0100208804002054
:10904C0050AB0008F90100207812002048AB000852
:04905C00A01200203E
:10906000F0B581B00125EE433046FF381B49096851
:109070004A6802404A6068024A6882434A602A029B
:109080000A600860164C2046FCF72AF92068002781
:10909000476206612046FCF7EBF80920FAF76EFEFE
:1090A000EA2010490F521048104901600920FAF7D0
:1090B00059FE0C4887850E4801680E610D4A0E4B1B
:1090C00013604F62FCF7D4F82120C000054A115A02
:1090D000491C11520948056001B0F0BD8805002007
:1090E00080110020FC0C00202C1300200100002027
:1090F000CC1100207C130020C58D0008C012002078
:10910000B0B5002901D0022523E013490A68821A6C
:10911000124C23689A421ED908601148402101F080
:109120000AFE454245410F490978002900D005460D
:109130000D480068A84202D10C490D4803E0A80080
:109140000C4908580C49AA000C4B985089582160CA
:10915000804705480560B0BD9813002098040020A2
:1091600000080050FB0100209404002050AB0008D0
:10917000F90100207812002048AB0008A812002056
:1091800010B50920FAF7FAFD074800F05BFF0B481D
:10919000012101800548064901600920FAF7E2FD36
:1091A00004480549016010BD210000202C13002057
:1091B000410300207C130020798D0008E60D00207B
:1091C000F0B581B0184800684168184E31404160E0
:1091D0000125690242688A4342602A0202600160F6
:1091E000134C2046FCF77CF8206800274762FF36C6
:1091F00006612046FCF73CF80920FAF7BFFDEA209B
:109200000C4E37520C480D4901600920FAF7AAFDAF
:1092100085204000315A491C3152094809490160F2
:109220000948056001B0F0BD88050020FFFEFFFF82
:1092300080110020FC0C00202C1300204500002091
:0C9240007C130020798D0008C012002073
:10924C00B0B5002902D00020C54323E013490A68B9
:10925C00821A134C23689A421ED908601148402187
:10926C0001F063FD454245410F490978002900D0C2
:10927C0005460E480068A84204DAA8000E490858B2
:10928C000E4901E00A490B48AA000D4B9850895829
:10929C002160804705480560B0BDC04628130020FA
:1092AC007C04002000080050FB0100207804002002
:1092BC0050AB0008F90100207812002048AB0008E0
:0492CC0098120020D4
:1092D000F0B581B00125EE433046FF381B490968DF
:1092E0004A6802404A6068024A6882434A602A0229
:1092F0000A600860164C2046FBF7F2FF2068002742
:10930000476206612046FBF7B3FF0920FAF736FDF6
:10931000EA2010490F521048104901600920FAF75D
:1093200021FD0C4887850E4801680E610D4A0E4BE1
:1093300013604F62FBF79CFF85204000054A115ADD
:10934000491C11520948056001B0F0BD8805002094
:1093500080110020FC0C00202C13002001000020B4
:10936000CC1100207C130020C58D0008C012002005
:1093700070B5002901D0042430E01A490A68821A25
:10938000194E33689A422BD90860184D402128465F
:1093900001F0D1FC04468021284601F0CCFC41427A
:1093A0004141134A1278002A00D0014660426041D0
:1093B000002A00D0204644000C430E480068844236
:1093C00002D10D490D4803E0A0000D4908580D4990
:1093D000A2000D4B985089583160804705480460C1
:1093E00070BDC046A0130020A0040020000800505B
:1093F000FB0100209C04002068AB0008F90100205C
:0C9400007812002058AB000888120020F1
:10940C00B0B50920FAF7B4FC0E4800F015FE0E4872
:10941C000E4901600920FAF79FFC124801210180D6
:10942C000B480C4901600C4C08210022204602F02C
:10943C0002F802212046002201F0FDFF07480849EE
:10944C000160B0BDA90000202C13002041030020B6
:10945C007C130020798D0008000400506C13002050
:08946C00F9010020E60D0020CB
:1094740070B50920FAF780FCEA20114E032131521D
:109484001048114901600920FAF76AFC0F48104995
:109494000160104C08210022204601F0D0FF022177
:1094A4002046002201F0CBFF2120C000315A491C84
:1094B400315209480949016009480121016070BD20
:1094C400FC0C00202C130020CD0000207C13002075
:1094D400798D0008000400506C130020F90100206D
:0494E400C012002092
:1094E800F0B581B00920FAF745FCEA20114F0224B3
:1094F8003C521148114901600920FAF72FFC104825
:1095080010490160104D08210022284601F095FFFE
:1095180028460221002201F090FF85204000395A98
:10952800491C395209480A4901600A480121016069
:1095380001B0F0BDFC0C00202C13002041010020DC
:109548007C130020798D0008000400506C13002063
:08955800F9010020C0120020FF
:10956000F0B581B01C48006841681C4E3140416034
:109570000125690242688A4342602A020260016052
:10958000174C2046FBF7ACFE206800274762FF36E9
:1095900006612046FBF76CFE0920FAF7EFFBEA2094
:1095A000104E37521048114901600920FAF7DAFBD2
:1095B0002120C000315A491C315285204000315AC7
:1095C000491C31520A480B4901600B480B490160A4
:1095D0000B48056001B0F0BD88050020FFFEFFFFCD
:1095E00080110020FC0C00202C130020B50100206D
:1095F0006C130020D98C00087C130020C58D000856
:04960000C012002074
:1096040070B5002906D0264800210170C8432549B9
:10961400086070BD24490A68821A244E33689A424D
:109624003CD90860224D4021284601F082FB0446C3
:109634008021284601F07DFB414241411D4A1278B8
:10964400002A00D0014660426041002A00D0204632
:1096540044000C43134D2868844207D1A100174AE3
:1096640018485050184A5158316015E00C48017898
:10967400012903D1A000114908580BE0002C01D0A6
:1096840001210170A1000C4840580C4A50500C4A6A
:1096940051583160002800D080472C6070BDC0460E
:1096A400BC13002080040020301300208404002018
:1096B40000080050FB0100207812002068120020EE
:0C96C40058AB0008F901002068AB00085A
:1096D000F0B581B00220C643F9F7B8FD0446174D36
:1096E000A88DC01EB04227D8154E3068201A1549E3
:1096F000884221D314480068211A144881421BD99A
:1097000013490968611A814216D91248FBF7E8FD2E
:109710000127F94310480268116134600021516249
:10972000FBF7A6FD0C20FAF71DFB43208000295A09
:10973000491C29520948076001B0F0BDFC0C00200B
:10974000E4120020E9030000640400201027000058
:10975000680400203411002004100020C0120020F2
:10976000F0B581B00220C043134CA18DC91E8142C7
:109770001ED81048006800281AD00125EE43F9F7DA
:1097800065FD0E490A6816610D4B18600027576287
:109790000846FBF76DFD0B4801680E614F62FBF751
:1097A00067FD43208000215A491C2152064805606C
:1097B00001B0F0BDDC120020FC0C00205010002095
:0C97C000E412002034110020C012002030
:1097CC000648006801210A020260490201604368F0
:1097DC001343436042680A43426070478805002087
:1097EC00F0B583B000252C462F461648066816495E
:1097FC000A680292036808680090002013492A4600
:10980C0001F0DBFE34190298C7196D1C1048854213
:10981C00EBD105463846294600F0E6FF0646104FC8
:10982C0078802046294600F0DFFF388082B2B3B240
:10983C000020084901F0C1FE07480849016003B047
:10984C00F0BDC046C8120020CC120020EEBC0008AF
:10985C0050C300001BBD00088C130020F901002030
:04986C00480D002083
:10987000F0B581B02E482F49FDF7D8FAF9F7E6FC8C
:109880000446F9F7E3FC001B2B4E0027B04215D22B
:109890003D46E81B294909680D18E817000F2818EC
:1098A0000711002026493A4601F08DFE0120F9F704
:1098B000D3FCF9F7CBFC001BB042EAD34E20214E7B
:1098C000305A3C1AE220305EC72802DC6E2060432A
:1098D00010E080B2C1084A2910D80A2141431A4831
:1098E000081880B2000919494143080C6E21081A72
:1098F00044432046642100F05DFF0446A5B26E207B
:109900006843642100F076FF40217052F4871048CC
:109910006043104900F04EFFB08783B200200E492B
:109920002A4601F050FE0D480D49016001B0F0BD1E
:1099300045BB0008EEB7000860EA0000CC1200202A
:1099400033BF0008FC0C002030F8FFFF3E0A000087
:10995000B80B0000FF0F000053BF00088C1300205D
:04996000F9010020E9
:10996400F0B581B00024104F25463E683B680020C6
:109974000E49224601F025FE7519641C0C488442E8
:10998400F3D10146284600F033FF0A49081A0A4970
:10999400488702B20020094901F013FE084809492A
:1099A400016001B0F0BDC046C412002015B8000823
:1099B40050C30000FF070000FC0C002040BD00085D
:0899C4008C130020F9010020C2
:1099CC00F0B583B00D46029001600C203F4906C5EE
:1099DC000021E86029616961A961E96129620126B8
:1099EC003703083D2C4680340998089A002B04D084
:1099FC00012B04D10321490202E0B10200E00F4621
:109A0C00AF602961511E4A1E91414903E96000F083
:109A1C00BDFE00272E4B3A4601F0ECFB00F09EFEFB
:109A2C0001906068002803D12770284600F044FE9E
:109A3C002420606028680168B14301602846FBF768
:109A4C00F3FD0128029C29D0A86A002802D02846E0
:109A5C0001F0A4F9B103286882680A438260F1031B
:109A6C0082688A43826001681A4A0A400260F105E2
:109A7C0042680A434260B10602680A430260FF2151
:109A8C00090642690A4001990A434261016831435F
:109A9C0001602846FBF7D0FE002801D0FFF7F0F854
:109AAC00206801F0B0FA002801D0FFF7E9F820682F
:109ABC00273432022146FBF7C7FF002804D00648A2
:109ACC000649FDF7E9F9FEE703B0F0BD00380140A7
:109ADC0000000C40FFFF00FCDFBF000866BD000863
:109AEC00F0B58DB005460268D16910680C90012064
:109AFC000A90000709900595843590680B9008072B
:109B0C00089048D00998431C0B9803400126370253
:109B1C003C4620340C9804401C433CD007407C420B
:109B2C007C41CF070A9F00D02746002F03D1166235
:109B3C00AC683443AC600B980640744274418F0798
:109B4C000A98074600D52746002F05D10224146237
:109B5C00AC6804272743AF60744274414E07064635
:109B6C0000D52646002E05D104241462AC680226CA
:109B7C002643AE60089800280DD55C1EA3410C98B6
:109B8C0084060A9C00D41C46012C04D108231362C1
:109B9C00AC681C43AC600126F00507900B050FD593
:109BAC000B9B0340B4060C980440E31808D0F30256
:109BBC00136220236B602B605A4B1E755A4C1E553A
:109BCC00049620200F460890074022D00B9B099842
:109BDC0003400C9C089804401C431AD06B68222B41
:109BEC0013D14523DB004F48C65804980402A64203
:109BFC000BD24C4CA019526A272682554A4A04981B
:109C0C00A054E258521CE25003E0936908241C4310
:109C1C00946180200E46069006400A9830D00B9A2C
:109C2C00079B1A400C9B069C2340134328D03D4AAB
:109C3C00136884241C59212C14D11C4656342288B8
:109C4C00002A0FD01A6802921A6D039212780194AE
:109C5C00029CA262039A521C1A65019B1A88521E1E
:109C6C001A8008E01A681368069CA34313601368F3
:109C7C0040241C4314602B4C23221201049BA3543C
:109C8C0040240C9B23405A425A41490600D51046A9
:109C9C0000280ED1254800210170059803681A6828
:109CAC00A2431A6041670899296001F059F92220F2
:109CBC006860A868002829D022236B60002F07D089
:109CCC000B98099901400C98089A104008431FD131
:109CDC00002E1BD00B99079801400C98069A104047
:109CEC00084313D026200F4E00213154059822270B
:109CFC0003681A68A2431A6041670899296001F049
:109D0C002FF96F6023200001049931540DB0F0BD80
:109D1C0005980068816908220A4382610020A860C6
:109D2C000DB0F0BDC00A002031020000E60A002090
:109D3C00F0B583B04521CB00C258052A3AD3019324
:109D4C002721415C00910290044627341046951E51
:109D5C001C4900261C4F03E0761CAE4219460CD061
:109D6C00A35D4B400721C94302E01346491CF3D2C3
:109D7C005A08DB07F9D07A40F7E7615D0219521EE9
:109D8C00127812025118C91A4A1E9141401C4242C3
:109D9C0042410A430298019B0CD10C49C98B009C8F
:109DAC000A1B51425141002C00D10121002901D044
:109DBC00022103E0C218002101751160084603B0AE
:109DCC00F0BDC046FFFF000001A00000FC0C00200D
:109DDC00F0B585B006468B208000049000273750E4
:109DEC002720335CFF242046283033540096351846
:109DFC00314627310122284601F0BDF9049971182A
:109E0C0002914521C90071180391049632462632FD
:109E1C000028214614D01449144B03E07F1C8742C0
:109E2C0021460CD0EC5D4C400721C94302E034467E
:109E3C00491CF3D26608E407F9D05E40F7E7210A23
:109E4C002C542B1859700C211170811C0298016034
:109E5C00049C20688AB22946FBF722FD0020039956
:109E6C000860207505B0F0BDFFFF000001A00000E8
:109E7C00F0B51E4C002B06D0E58B9D4203D08621FD
:109E8C0081540B211BE04D790B791B025B191E468B
:109E9C007E3E7D27FF43BE4203D88321815403219C
:109EAC000DE0CE788978090289195B181E468C3E24
:109EBC008B27FF43BE4206D8832181540221101800
:109ECC004170901CF0BD0326865486186D00757089
:109EDC004D00641985186678AE702678EE70A41C57
:109EEC00921C491C9942F5D3901CF0BDFC0C00202F
:109EFC00F0B51D4C002B08D0E58B9D4205D086217A
:109F0C008154531C02240B212AE0CB788D782D022E
:109F1C00ED188B2D09D28D26B600059FBE1937681A
:109F2C007F5D022F07D0002F09D186218154531C4D
:109F3C0002210C4614E076683688002EF5D06D00B0
:109F4C0066190F7977704E796655062484548418F7
:109F5C00A370002363700B79E370131D49790524FA
:0C9F6C00C154A018F0BDC046FC0C002041
:109F7800F0B585B00490304D022401200390002BE9
:109F880006D0E88B984203D00B26862310464BE078
:109F98004F7908790002C01905467C3D7A23DE43D3
:109FA8009023B54202D2032610463DE00297CD78B1
:109FB8008C780194240200956719C51928468C38B5
:109FC8008A24E4430226A042104634462CD316467F
:109FD8008D2080000A9A13187800174A1418C91D92
:109FE80008E00878607048782070A41C891C7F1CE1
:109FF800AF420AD21868C05D0028F6D00228F0D116
:10A00800586800880028ECD1EFE710203246049900
:10A01800885588190099817001994170F01C0524B0
:10A02800042103910023029E04990B54039880187D
:0CA038000E54A01805B0F0BDFC0C002078
:10A04400002801D0014908607047C0460813002069
:10A0540000B583B00D484168012211434160416855
:10A06400114002910299110702680A4302600068D4
:10A07400084001900198F9F709F90220F9F7FCF872
:10A0840003204002F9F70AF903B000BD3C10024076
:10A09400FAF73CFF054C064D0221204601F0D7F9A2
:10A0A4000020294600F0FCFCF6E7C04600040050FE
:04A0B40037BB0008AE
:10A0B8000020064900F0F2FC0549002000F0EEFC03
:10A0C800044C0221204601F0C0F9FAE7E3BF00087A
:08A0D800EBBF0008000400507A
:10A0E00080B50248FBF716F980BDC046501000202D
:10A0F00080B50248FBF70EF980BDC0460410002071
:10A1000080B50248FBF706F980BDC046CC1100209F
:10A1100080B50248FBF7FEF880BDC04680110020E4
:10A1200080B50248FBF7F6F880BDC0463411002028
:10A1300080B50248FBF7EEF880BDC046E81000206D
:10A14000B0B50446FBF7CCF820682749884216D002
:10A1500026490968884221D0254D296888421CD0AB
:10A160002449884223D02449884223D02349884265
:10A1700013D1FFF72BFB2046FBF7B2F8B0BD214C03
:10A180000125A5852548FFF75DFFEA2025521E48D9
:10A19000234901601E4823490160B0BD19480221CE
:10A1A00081851D480268002001219047B0BD1448F8
:10A1B0000121F1E7FEF738FCEA20124900240C5295
:10A1C0001148124A02608C851148124901602846E4
:10A1D000FBF786F80120C043296808614C622846D5
:10A1E000FBF746F8B0BDC046001000400410002048
:10A1F000CC110020004801400044014000400140D3
:10A20000F4120020FC0C00202C1300200100002080
:10A210007C130020C58D00089C130020D501002070
:08A2200041030020E58D000858
:10A2280070B516490868164A13684340154C2268E9
:10A238001A40D5432560144C26681E406E4026609F
:10A248005A40324050400860024010490B6813439E
:10A258000B600C21014005D00D480268521E0260B7
:10A2680004D070BD0A480C49016070BD64220260C8
:10A27800084802680A43026070BDC046E812002020
:10A28800100C005000130020FC120020F0120020D7
:0CA29800F8120020EC1200205F0900000A
:10A2A40004490968884304490A68104042400A6026
:0CA2B4007047C046E8120020F0120020A5
:10A2C00005490A68104042400A6004490A68104083
:10A2D00042400A607047C046EC120020F012002095
:10A2E00030B587B0154800248461E1430125AA07F1
:10A2F00014C0046041608460069405940494019441
:10A30000083800F01FFD002801D0FEF7BFFC28032D
:10A3100003900A4803A9FBF7AFF8002801D0FEF725
:10A32000B5FC0294009405486946FBF745F90028FE
:10A3300001D0FEF7ABFC07B030BDC0469C1000203A
:10A3400010B584B00E48002484610E49F9220E4BEA
:10A35000036042608460C160029400F0F3FC002856
:10A3600001D0FEF793FC03940194054801A9FBF783
:10A3700023F9002801D0FEF789FC04B010BDC046C7
:0CA3800050100020FFF900000010004009
:10A38C0010B584B00E48002484610E49F9220E4B9E
:10A39C00036042608460C160029400F0CDFC002830
:10A3AC0001D0FEF76DFC03940194054801A9FBF75D
:10A3BC00FDF8002801D0FEF763FC04B010BDC046C8
:0CA3CC0004100020FFF900000014004005
:10A3D80010B5094800218161084A6323084C0460CC
:10A3E80043608160C260016100F0A8FC002801D0D0
:10A3F800FEF748FC10BDC046CC110020FFF9000054
:04A4080000200040F0
:10A40C0010B588B0154800241549164A14C00460CC
:10A41C0041608460C46004610794069405940294BE
:10A42C00083800F089FC002801D0FEF729FC012037
:10A43C0000030490094804A9FBF718F8002801D080
:10A44C00FEF71EFC03940194044801A9FBF7AEF837
:10A45C00002801D0FEF714FC08B010BD80110020BC
:08A46C00FFFF00000040014069
:10A4740010B509480021094A094B0A4C046043609D
:10A484008160C26001614161816100F059FC002872
:10A4940001D0FEF7F9FB10BD34110020FFF90000D4
:08A4A4005FEA000000440140E2
:10A4AC0010B509480021094A094B0A4C0460436065
:10A4BC008160C26001614161816100F03DFC002856
:10A4CC0001D0FEF7DDFB10BDE81000200F270000C7
:08A4DC00FFF9000000480140F7
:10A4E40010B58EB0044601A8001D302100F006FB13
:10A4F40020684D49884223DD4C4988423BDC4E4963
:10A5040088424FD04D49884200D08AE00124A005FA
:10A51400019001A8FAF710FD002801D0FEF7B4FB62
:10A52400200449490A6802430A600968014000910D
:10A534000098142000210A46F9F7F2FB14206EE07B
:10A5440001218A0790423ED03D49884246D03D4988
:10A55400884266D13C48001F0168202211430160F3
:10A564000068104000900098122003210022F9F79F
:10A57400D7FB122053E02E49884240D02D4988420F
:10A584004FD10120800430490A6802430A600968F7
:10A59400014000910098162003210022F9F7C0FB26
:10A5A40016203CE00120C00327490A6802430A60E0
:10A5B4000968014000910098132003210022F9F753
:10A5C400AFFB13202BE02048001F02680A430260FF
:10A5D40000680840009000980EB010BD1A48001F93
:10A5E4000168102211430160006810400090009837
:10A5F400112003210022F9F793FB11200FE0012021
:10A60400400411490A6802430A6009680140009144
:10A614000098152003210022F9F782FB1520F9F791
:10A624009FFB0EB010BDC046FF1F0040FF4301401A
:10A634000044014000480140002000400040014027
:0CA64400001000400014004040100240D4
:10A65000B0B51A4800210C22194B01624162816297
:10A66000036001239C021B03E1256D0245608360AA
:10A67000C160046142618161C1610A460B46FBF71A
:10A680004DFC002801D0FEF701FB0C480021FBF730
:10A690008BFC002801D0FEF7F9FA08480021FBF7EF
:10A6A000C3FC002801D0FEF7F1FA044800F0B1FC29
:10A6B000002801D0FEF7EAFAB0BDC046BC0E00206B
:04A6C000003801401D
:10A6C400F0B595B0044603A808302C2100F016FA22
:10A6D40020682249884201D015B0F0BD02250495B6
:10A6E4000127039703A8FAF727FC002801D0FEF7F7
:10A6F400CBFAB8031A49CA680243CA60CA6802405E
:10A70400109210980868384308600868384002902E
:10A714001497002413941294119509204002109068
:10A72400029805200195050710AE28463146F9F731
:10A734002FFF14971394129701981190B802109058
:10A7440028463146F9F724FF1B2003210022F9F79C
:10A75400E7FA1B20F9F704FB15B0F0BD00380140FF
:04A76400341002406B
:10A768004A0010D2520D03231B02FF33D21A0AD417
:10A7780052421F3209D4400DC90208430123DB07A6
:10A788001843D040704700207047D0177047C04624
:10A7980042221201033A010007D002D4013A0018FC
:0CA7A800FCD51205C30A40059918704743
:10A7B400CA1751408B1A17D0C1174A4094464840D3
:10A7C400411A48081A0000E052008242FCD90020D5
:10A7D40000E05208914200D3891A40419A42F8D1CC
:10A7E40062465040801A704710B500F075F810BDED
:10A7F4000A0015D00300400800E052008242FCD950
:10A80400002000E052089B1A06D340418A42F9D145
:10A81400704752089B18F8D200188A42F9D1704741
:08A8240010B500F059F810BD59
:10A82C0038B504004D42FFF7DFFF4543611938BDD1
:10A83C00002B09D1002907D110B51100FFF7F0FF4B
:10A84C000A000021002310BD70B400240125ED077F
:10A85C00002B07D1002905D0834203D2130000221C
:10A86C002C0000250026A419994200D1904212D93F
:10A87C0092185B4103D2EE076D086408F3E7DE071C
:10A88C005B08520892190126F6079B1903E0DE07B4
:10A89C005B0852089219801A994103D364416D41A7
:10A8AC00F5D30FE024196D410AD2DE075B0852087C
:10A8BC00921980185941F5D364416D41E7D301E0F9
:10A8CC008018594102000B002000290070BC704711
:08A8DC00002000217047C04676
:10A8E40003230F480F4A036143610F4B8261C36125
:10A8F4008023DB000362002383624362C362026637
:10A904000A4A426610228266094A0367C36643679D
:10A914001178013AC1540133102BF9D17047C04664
:10A92400140E002090AB0008C0060020581200202E
:04A93400ABAB0008C1
:10A93800F8B54746CE46C56883680400406899461E
:10A948005B1B80B50E00170098464019934207D943
:10A9580000F0CAF8ED19E560C0BCB946B046F8BDCC
:10A968001A0000F0C1F84B463100ED19ED1A2A0023
:0CA978006068414400F0B8F8EDE7C0460C
:10A98400F8B54746CE46002380B588460700160032
:10A994009946C56884681BE0013B5B1B641BB44299
:10A9A40000D934009C4200D91C007868220041463A
:10A9B400401900F09BF82D19A144A044361BBC6833
:10A9C400631B5A1E93415B421D40FD60002E06D05E
:10A9D4003B699D42E0D3013B1B195B1BDEE7484604
:08A9E400C0BCB946B046F8BD45
:10A9EC0070B50600431C5C00E4181D4BE400E01835
:10A9FC007400A419E4001B19DC6A1500012C06D0A4
:10AA0C00022C1FD0002C10D00024200070BD9A6A9C
:10AA1C005C6AA2421FD9013A121B2C00954200D944
:10AA2C0014002200FFF782FFEFE79A6A5E6AB242D7
:10AA3C000CD9013A961BB542E7D82A00FFF776FFEE
:10AA4C002C00E2E7FFF798FF0400DEE71B6AD21840
:10AA5C00013A961BEFE71B6AD218013A121BDCE78E
:04AA6C00140E0020A4
:10AA7000F8B50B4B04001B780D001600002B0CD012
:10AA8000EFF31087012181F31088320029002000A4
:10AA9000FFF7ACFF87F31088F8BDFFF723FFEFE760
:04AAA000140E002070
:10AAA400F8B5050008000C0000F018F80A4B060081
:10AAB4001B78002B0CD0EFF31087012181F3108851
:10AAC400320021002800FFF78FFF87F31088F8BDBC
:0CAAD400FFF706FFEFE7C046140E00205D
:10AAE000411C02780130002AFBD1401A7047C04651
:10AAF000002A03D0013A8B5C8354FBD17047C046D7
:10AB000000220B0011001A00002A02D0013A8154E1
:04AB1000FCD17047BD
:10AB14000000000004000000020000000800000023
:10AB2400004B0000650001000100E8030000000084
:10AB34000000C80011014C042602EE02DC05E0010D
:04AB4400000000000D
:08AB48000A000000B80B000038
:08AB5000010000006400000098
:10AB58000A000000B80B0000B80B0000B80B00009A
:10AB680001000000640000006400000064000000B0
:10AB7800034C206804348047FBE7FCF7ADF9FEE797
:04AB880000C0000801
:04AB8C00D1300008BC
:09AB90005465726D696E616C0080
:03AB99003A20005F
:10AB9C0000000000000054545220524547474553D2
:01ABAC0000A8
:10ABAD004465766963652049443A20756E6B6E6F16
:03ABBD00776E00B0
:02ABC000FEE7AE
:02ABC200FEE7AC
:02ABC400FEE7AA
:02ABC600FEE7A8
:02ABC800FEE7A6
:02ABCA00FEE7A4
:02ABCC00FEE7A2
:02ABCE00FEE7A0
:02ABD000FEE79E
:02ABD200FEE79C
:02ABD400FEE79A
:02ABD600FEE798
:02ABD800FEE796
:02ABDA00FEE794
:02ABDC00FEE792
:02ABDE00FEE790
:02ABE000FEE78E
:02ABE200FEE78C
:02ABE400FEE78A
:02ABE600FEE788
:02ABE800FEE786
:02ABEA00FEE784
:02ABEC00FEE782
:06ABEE00F8F767FAC1E769
:0AABF40080B5806A00F055F880BDBE
:10ABFE0080B5806A816D40220A438265C16D042250
:0AAC0E000A43C26500F047F880BD5C
:10AC1800F0B581B004465420205C012801D10225FA
:10AC280038E026465436012737702046F8F76CFC82
:10AC3800054600282CD1206D2521415C022911D11F
:10AC4800F9F7E6FA00280DD00546A06D402101432A
:10AC5800A165206841681022914341602046F8F7B9
:10AC680081FC11E020684168102291434160204630
:10AC7800F8F778FC0546002806D1FF200230A16DC0
:10AC88008143481CA06500252068C168B943C1609C
:0AAC980000203070284601B0F0BD26
:02ACA2007047F9
:02ACA4007047F7
:02ACA6007047F5
:10ACA80070B54279012A01D1022070BD02230371D7
:10ACB80010240C4001221546A540046826682E433E
:10ACC8002660256800290ED01E468E401F214904A3
:10ACD8000D40B54202D1616819436160002141719C
:10ACE8000271002070BD3E210D40022D1346F2D0A6
:02ACF800F4E77F
:10ACFA0010B581B00024009400680090002903D0A8
:10AD0A0000981018143002E00098101808300090CB
:0AAD1A0000980360002001B010BD96
:10AD240010220A401F2191400068806B0840D040E7
:02AD3400704766
:0AAD360000690840411E8841704783
:02AD400070475A
:02AD4200704758
:10AD4400F0B581B0002823D0044605463C350746BB
:10AD54003E37064644366878002803D128702046DA
:10AD6400FFF7BEFB0220687001CC2146FAF7E8F930
:10AD74000120307138707870B870F870387178715B
:10AD840030707070B070F0706870002001B0F0BD69
:06AD9400012001B0F0BD3A
:02AD9A00704700
:02AD9C007047FE
:02AD9E007047FC
:02ADA0007047FA
:02ADA2007047F8
:02ADA4007047F6
:02ADA6007047F4
:10ADA80030B5816ACA070CD18A0714D44A071CD463
:10ADB8000A0724D4CA062CD48A0634D44A063CD4BA
:10ADC8004CE00122520403685C689443C26A22433F
:10ADD8005A608A07EAD50122120403685C68944322
:10ADE800026B22435A604A07E2D5012292040368A3
:10ADF8005C689443426B22435A600A07DAD5012201
:10AE0800D20303685C689443826B22435A60CA0683
:10AE1800D2D50122120303689C689443C26B224373
:10AE28009A608A06CAD50122520303689C68944333
:10AE3800026C22439A604A0610D501221305026863
:10AE480054689C43456C2C4354609D4206D10323AF
:10AE58005B0554689C43836C23435360090607D5FC
:10AE68000121C904026853688B43C06C18435060C1
:02AE780030BDEB
:10AE7A00F0B585B0049316460F4604460368D969AF
:10AE8A003940C91B4A424A410020B24242D102908B
:10AE9A002146803101910A9D01210091C802039047
:10AEAA0006E0D9693940C91B4A424A41B24230D107
:10AEBA00691CF6D0F8F7C5F9002D2DD00499401A6F
:10AECA00A84229D8236819684907EAD5D969039895
:10AEDA000142E6D01862EFF31080009D85F31088D6
:10AEEA000D214901226813688B43136080F310888F
:10AEFA00EFF3108085F3108821688A68AA438A6074
:10AF0A0080F310882020019A5060906010460C301F
:10AF1A001EE0029805B0F0BDEFF31080009D85F3A6
:10AF2A0010880D214901226813688B43136080F34E
:10AF3A001088EFF3108085F3108821688A68AA4385
:10AF4A008A6080F310882020019A506010460830E9
:0EAF5A000021117020210160032005B0F0BD20
:02AF6800704730
:02AF6A0070472E
:02AF6C0070472C
:02AF6E0070472A
:10AF700070B5026801465C318B88CC6A222C0DD1F9
:10AF8000526A1A40836D1A704A88521E4A80826D36
:10AF9000521C82654A88002A05D070BD906908213C
:10AFA0000143916170BDEFF31083012282F3108899
:10AFB0000924640105682E68A6432E6083F3108877
:10AFC000EFF3108382F310880468A5689543A560A9
:10AFD00083F310882023CB6200230367C46E012C07
:10AFE00014D1C366EFF3108382F3108804682568D8
:10AFF00010229543256083F310880368DC69E4061A
:10B0000000D51A620988FFF7B0FF70BDFFF7AFFFE8
:02B0100070BD11
:10B0120030B58021415C012901D1022030BD0246B8
:10B0220080322421516001680B680C680125AC4311
:10B032000C606C07A3430B60002141661170202055
:06B042005060002030BD4B
:10B0480010B5044642688368581C904202D993425E
:10B0580009D010BD2268D154A060E168491CE160A4
:10B0680062689042F5D121682069FFF7FDFCA1686C
:10B07800884202D10020A06010BD0020C043E060DB
:02B0880010BDF9
:06B08A00F920C000704730
:10B09000F0B581B0002816D014460D460646FF27AD
:10B0A0004E3701222846214600F0CBF93846F8F702
:10B0B000D3F800222846214600F0C3F93846F8F7B5
:0AB0C000CBF8761EEDD101B0F0BD13
:10B0CA00F0B581B01D4614460F460646F8F7B9F8A2
:10B0DA003A68AA420BD22368022B1CD0054609996A
:10B0EA000898012B07D0002B03D101220BE0002086
:10B0FA00386001B0F0BD069B52009A5A3368EB1AC9
:10B10A009342F6D9002200F097F935602068401C76
:10B11A00206001B0F0BD034607985100405A3168DB
:10B12A00591A8142E5D93360002020603868401CF2
:02B13A00DEE74E
:10B13C00B0B582B01D4613460A4604460B2001905A
:10B14C00022B01D3022000E001200090204629466A
:10B15C00FEF736FC2620002121548D208000069A13
:10B16C002250A184E161218420181C34A17107991B
:06B17C00416002B0B0BD0D
:10B18200B0B582B04C78069D102C07D0062C0AD0A0
:10B19200032C0DD1FEF771FE02B0B0BD0095FEF793
:10B1A200EAFE02B0B0BD0095FEF7A7FE02B0B0BD48
:10B1B20080214C408454801801214170901C02B0BF
:02B1C200B0BD1E
:02B1C4007047D2
:02B1C6007047D0
:10B1C80008D1002806D1F54204D801D3002A01D1BC
:10B1D8006D0D09D10020C143090DC904F0BDF9D195
:10B1E8001242F7D1640DF5D00020C1434905490842
:10B1F800A6E000206146F0BDF0B50127FF070E006C
:10B208005E403E40B446BE0A4C18DD18F442D7D220
:10B21800F542E4D2640DECD06D0DEAD06419C90290
:10B228003943460DC0023143DB023B43DB0A10B40D
:10B238008E4685B297B26F43140C6C433E0CA4192A
:10B24800260C2404BFB227439CB26C43A419190CE2
:10B258006943250CA4B249190D04090C6419000CA2
:10B2680095B245433E0C76193743BFB2360C150CE0
:10B278004543AD19A6B2240CAD192E0437432E0C44
:10B2880036199DB24543AD19ACB22E0C89191D0C67
:10B2980045436D182E04290C3443704680B295B28C
:10B2A80045433E0C76193743BFB2360C150C45435F
:10B2B800AD19A6B2AD19240C2E0437432E0C36193D
:10B2C8009DB24543AD19ACB22E0C89191D0C4543EE
:10B2D8006D182E043443290C75462D0C90B2684322
:10B2E8003E0C80190604BFB23E43070CA0B23F18BB
:10B2F800120C6A43D019020C80B2240CA4189AB21A
:10B308006A43121914042043120C89181B0C6B434E
:10B31800C91810BC01273D05294203D1B61940417F
:10B328004941013CFF077D0D013D641B0BDB6D00AE
:10B33800AC4209DA240500254208BE416841614152
:0AB3480066463143F0BD54E74EE7BE
:10B35200B0B504465420205C012801D10220B0BDC2
:10B3620025465435012028702046F8F7D0F80028E9
:10B372000BD12046F8F7F9F8002806D1FF20023059
:10B38200A16D8143481CA065002000212970B0BD39
:10B39200B0B50146806A836D826D5024234206D087
:10B3A200D20610D4006D426B08469047B0BD012111
:10B3B2004B021A4382650268D3681B059B0F05D0B6
:10B3C200FFF76EFCB0BDFFF76CFCB0BD837E002BB7
:10B3D200F6D113681B07F3D593685B070AD40346BB
:10B3E200583354680C25AC435460FF2402341A6865
:10B3F200A24306E0826D20231343836503465C3338
:0CB40200C26D0A431A60FFF74BFCB0BD9E
:0CB40E000068B42141587F2008407047BE
:10B41A0010B500280ED004460079002803D16071C7
:10B42A002046FBF74EFA02202071002020610121FC
:08B43A00217110BD012010BDBD
:10B44200002A02D01822815070472822815070476A
:10B4520042690B4693430A401104C918816170473F
:10B4620030B584214158212904D1014656318A8AB6
:10B47200002A03D130BD521E1304FBD00B88002BCF
:10B482000CD00368DC692406F5D5046D25789D622D
:10B49200631C03650B885B1E0B80ECE7EFF31081E6
:10B4A200012282F31088D3050468A5689D43A56034
:10B4B20081F31088EFF3108182F31088006802682C
:0CB4C20040231343036081F3108830BD69
:10B4CE0030B58421415821290DD1014656310A88C3
:10B4DE00002A09D00268036D1C7894625A1C02651A
:10B4EE000888401E088030BDEFF31081012282F3E0
:10B4FE00108803681C688025AC431C6081F310889B
:10B50E00EFF3108182F31088006802684023134322
:08B51E00036081F3108830BDC9
:10B5260070B5026801465C318B88CC6A222C0CD13E
:10B53600526A1340826D13804B885B1E4B80921CAF
:10B5460082654A88002A05D070BD906908210143AA
:10B55600916170BDEFF31083012282F310880924F4
:10B56600640105682E68A6432E6083F31088EFF306
:10B57600108382F310880468A5689543A56083F359
:10B5860010882023CB6200230367C46E012C14D1DC
:10B59600C366EFF3108382F31088046825681022CF
:10B5A6009543256083F310880368DC69E40600D5BB
:10B5B6001A620988FFF7D6FC70BDFFF7D5FC70BD8F
:10B5C60082B000B581B00292039302AA00926A4645
:0CB5D600FAF767FD01B002BC02B00847A4
:04B5E200007D704731
:10B5E600010002000400060008000A000C0010001A
:08B5F60020004000800000016C
:10B5FE00547279696E6720746F207265737461720C
:03B60E00742E0097
:10B6110043616E6E6F74207265616420737461742E
:10B6210069737463616C20646174612066726F6D0B
:0FB6310020464C415348206D656D6F72792100A2
:10B640004144432063616C6962726174696F6E206A
:07B650006572726F722100A8
:10B657005374617274696E6720566563746F7220E4
:10B667005461626C6520636F7079696E67206672DA
:10B677006F6D20464C41534820746F2052414D2E28
:03B687002E2E0064
:10B68A004D6F646520302069732073656C6563743F
:10B69A0065642E204175746F2D7265636F6E6E65D9
:0BB6AA006374206973204F46462E0099
:10B6B5004D6F646520312069732073656C65637413
:10B6C50065642E204175746F2D7265636F6E6E65AE
:0BB6D5006374206973204F46462E006E
:10B6E0004D6F646520322069732073656C656374E7
:10B6F00065642E204175746F2D7265636F6E6E6583
:0BB700006374206973204F46462E0042
:10B70B004D6F646520332069732073656C656374BA
:10B71B0065642E204175746F2D7265636F6E6E6557
:0BB72B006374206973204F46462E0017
:10B736004D6F646520342069732073656C6563748E
:10B7460065642E204175746F2D7265636F6E6E652C
:0BB756006374206973204F46462E00EC
:10B761004D6F646520352069732073656C65637462
:10B7710065642E204175746F2D7265636F6E6E6501
:0BB781006374206973204F46462E00C1
:10B78C00555020627574746F6E206973206C6F6EE7
:0BB79C00672D707265737365642E00EA
:0BB7A70056613A20253664206D5600E4
:0BB7B20056623A20253664206D5600D8
:0BB7BD004441435F413A202534640002
:0BB7C8004441435F423A2025346400F6
:03B7D3004F5000D4
:03B7D600434C00E1
:03B7D900424100EA
:03B7DC00414200E7
:03B7DF00257300CF
:03B7E2004F5400C1
:03B7E5004F4300CF
:03B7E8004F4C00C3
:03B7EB004C4200CD
:10B7EE0043757272656E742063616C6C696272610E
:10B7FE0074696F6E2073657175656E636520737401
:07B80E0061727465642E00F5
:10B81500095B2534645D2053616D706C6564207629
:0BB82500616C75653A202534640A0050
:0BB8300048414C206572726F722100CD
:10B83B0053415645204C4F434B2D4B455920434FBD
:07B84B004D4D414E442E005B
:10B8520043616E6E6F7420726573746F72652064DB
:10B86200656661756C742073657474696E677320A4
:10B8720066726F6D20464C415348206D656D6F7244
:03B8820079210029
:02B885000A00B7
:10B887004465766963652049443A2053544D333201
:10B8970047304231206F722053544D333247304383
:02B8A70031006E
:10B8A9004465766963652049443A2053544D3332DF
:10B8B90047303731206F722053544D333247303877
:02B8C90031004C
:10B8CB004465766963652049443A2053544D3332BD
:10B8DB0047303531206F722053544D333247303659
:02B8EB0031002A
:10B8ED004465766963652049443A2053544D33329B
:10B8FD0047303331206F722053544D33324730343B
:02B90D00310007
:10B90F004672656520737061636520666F72206390
:10B91F006F66696775726174696F6E20696E2066F4
:10B92F00616B6520454550524F4D3A202575206279
:06B93F00797465730A0033
:10B945004D41585F504F535349424C455F4449461A
:10B95500465F544F5F4D4541535552453A20257535
:02B965000A00D6
:10B9670043616E6E6F742073746172742041444337
:0EB9770020696E20444D41206D6F64652100F3
:10B9850043616E6E6F7420636F70792056656374C2
:10B995006F72205461626C652066726F6D20464C33
:10B9A50041534820746F2052414D2120444D412080
:0EB9B5006973206E6F742072656164792100E1
:10B9C30043616E6E6F742066696E69736820636F7E
:10B9D3007079696E6720566563746F722054616273
:10B9E3006C652066726F6D20464C41534820746F1E
:06B9F3002052414D21002D
:10B9F9004D6F646520302069732073656C656374CD
:10BA090065642E204175746F2D7265636F6E6E6566
:0ABA19006374206973204F4E2E0065
:10BA23004D6F646520312069732073656C656374A1
:10BA330065642E204175746F2D7265636F6E6E653C
:0ABA43006374206973204F4E2E003B
:10BA4D004D6F646520322069732073656C65637476
:10BA5D0065642E204175746F2D7265636F6E6E6512
:0ABA6D006374206973204F4E2E0011
:10BA77004D6F646520332069732073656C6563744B
:10BA870065642E204175746F2D7265636F6E6E65E8
:0ABA97006374206973204F4E2E00E7
:10BAA1004D6F646520342069732073656C65637420
:10BAB10065642E204175746F2D7265636F6E6E65BE
:0ABAC1006374206973204F4E2E00BD
:10BACB004D6F646520352069732073656C656374F5
:10BADB0065642E204175746F2D7265636F6E6E6594
:0ABAEB006374206973204F4E2E0093
:10BAF500555020627574746F6E206973207072657D
:06BB0500737365642E005D
:02BB0B004E00EA
:06BB0D00523A20257300EE
:02BB13000A0026
:10BB150043616E6E6F742073617665206461746134
:10BB250020696E20464C415348206D656D6F7279D2
:02BB35002100ED
:0EBB37004E4D49204552524F522121210A0005
:05BB45004D41494E00D6
:10BB4A0043616E6E6F742073746172742054494D30
:05BB5A004552322100FC
:05BB5F001B5B324A00EF
:10BB640050726F6772616D20737461727465642EB4
:01BB740000D0
:10BB750043505520467265713A20257520487A0A4A
:01BB850000BF
:10BB860043616E6E6F74207265616420636F6E66CA
:10BB9600696775726174696F6E2066726F6D204693
:0DBBA6004C415348206D656D6F7279210090
:10BBB300257325733A204144432043616C696272C3
:10BBC3006174696F6E2076616C75653A2025750A1C
:01BBD3000071
:10BBD40043616E6E6F742073746F7020414443210F
:01BBE4000060
:10BBE50025733A204441432043616C696272617454
:10BBF500696F6E2076616C756520666F722063686B
:0DBC0500616E6E656C20313A2025750A00D5
:10BC120025733A204441432043616C696272617426
:10BC2200696F6E2076616C756520666F722063683D
:0DBC3200616E6E656C20323A2025750A00A7
:10BC3F0049742069732074696D6520746F20736176
:10BC4F00766520737461746973746963616C2064C1
:10BC5F0061746120696E20466C617368206D656D3B
:05BC6F006F72792E0048
:10BC7400496C6C6567616C204D6F64652069732045
:10BC840073656C65637465642E2044656661756CC8
:10BC940074204D6F646520342069732073656C656E
:10BCA400637465642E204175746F2D7265636F6EC5
:0DBCB4006E656374206973204F46462E00B4
:05BCC10025732573004E
:09BCC600493A20253564204100B3
:09BCCF004F56503A202531730054
:09BCD8004C56503A20253173004E
:0DBCE100543A202532642E256420B0430023
:10BCEE00095B2534645D2053616D706C656420764C
:10BCFE00616C7565733A20492B203D2025367520E1
:0DBD0E00202020492D203D202536750A00FB
:10BD1B0009094F66667365742076616C7565733AB5
:10BD2B0020492B203D20257520202020492D203D0A
:05BD3B002025750A003F
:10BD400009094F66667365742076616C75653A20E3
:05BD50002534640A0027
:10BD5500556E6B6E6F776E20636F6D6D616E6421CE
:01BD650000DD
:0DBD66005553415254206572726F722100D6
:08BD73000101010307010000BA
:08BD7B000804020408010101A3
:10BD8300303132333435363738394142434445460E
:08BD93001B5B323B33326D00F3
:08BD9B001B5B323B33336D00EA
:08BDA3001B5B323B33316D00E4
:10BDAB0025733A205265766973696F6E206E756DD7
:0CBDBB006265723A2030782534580A0086
:10BDC7004672656520737061636520666F722073C4
:10BDD70074617469737469637320696E2066616B3B
:10BDE7006520454550524F4D3A202575206279749C
:04BDF70065730A0066
:10BDFB00435055207370656564206973206E6F74B2
:08BE0B002036344D487A210075
:10BE13004669727374207374617274212057726956
:10BE230074696E672064656661756C7420636F6EF8
:0CBE330066696775726174696F6E2100AA
:08BE3F001B5B313B33326D0047
:10BE4700566563746F72205461626C652068617314
:10BE5700206265656E20636F706965642066726F26
:10BE67006D20464C41534820746F2052414D2E009F
:10BE7700496C6C6567616C204D6F64652069732040
:10BE870073656C65637465642E2044656661756CC3
:10BE970074204D6F646520342069732073656C6569
:10BEA700637465642E204175746F2D7265636F6EC0
:0CBEB7006E656374206973204F4E2E00EE
:10BEC300444F574E20627574746F6E2069732070EF
:08BED3007265737365642E00B3
:08BEDB001B5B323B33306D00AC
:08BEE3002573207C202573006B
:0CBEEB005661623A20253464206D560038
:0CBEF7005662623A20253564206D56002A
:10BF03001B5B323B33316D591B5B313B33326D006D
:08BF13001B5B313B33316D0073
:08BF1B001B5B313B33366D0066
:08BF2300434847202D203100A6
:08BF2B00434847202D2030009F
:10BF33000909566F6C746167652D64726F702041D7
:10BF430044432076616C75653A202535642E0A00DA
:10BF530009090946696E616C20766F6C74616765C7
:10BF63002D64726F70204144432076616C75653A8D
:10BF7300202534752E2046696E616C20766F6C74B3
:10BF83006167652D64726F702076616C75653A2008
:08BF9300253375206D560A00EC
:10BF9B0043616E6E6F742073617665206E657720DA
:10BFAB00534E20696E20464C415348206D656D6F92
:04BFBB007279210076
:10BFBF0043616E6E6F742073746172742054494DB7
:10BFCF00313720696E20495352206D6F646521000F
:04BFDF004D4F44007E
:08BFE3001B5B313B33316D00A3
:10BFEB00486172646661756C74204552524F5221E0
:04BFFB0021210A00F6
:01BFFF00FF42
:10C00000C9E50008370500207E0E0000C9E50008DC
:10C01000B613002003000000C9E50008BA13002091
:10C0200003000000C9E50008BE1300200300000063
:10C03000C9E50008C213002003000000C9E500089C
:10C04000C813002001000000C9E50008CC1300203F
:10C0500001000000C9E50008D01300200100000025
:10C06000C9E50008D21300200C000000DBE5000841
:10C070000000002090C0000837050000DBE5000844
:10C0800000600020C7C500080020000083AB000846
:10C0900006480068C16A0E2900D90F39026B816019
:10C0A0000E2A00D90F3A42617047C046EC050020C5
:10C0B00006480068C26A06498A4200D20F32036B02
:10C0C00082608B4200D20F3343617047EC05002041
:10C0D000F10F000006480068C16A0E2900D90F3927
:10C0E000026B81600E2A00D90F3A42617047C04648
:10C0F000EC05002006480068C26A06498A4200D260
:10C100000F32036B82608B4200D20F334361704762
:10C11000EC050020F10F000006480068C16A0E29F6
:10C1200000D90F39026B81600E2A00D90F3A4261A3
:10C130007047C046EC05002006480068C26A064900
:10C140008A4200D20F32036B82608B4200D20F33DF
:10C1500043617047EC050020F10F0000F0B517486F
:10C160000068C16A3A22164B9C5E164D2A68121965
:10C17000154EB242154F03DA0E2911D8002310E0F4
:10C180000123B9421F4600D300272D682C19B44261
:10C1900000DC00233B400F220C4F002B05D105E0B3
:10C1A00001230E22D243002B00D089188160016B3D
:10C1B000B94200D20F314161F0BDC046EC0500200C
:10C1C000FC0C0020C412002098090000F10F0000B0
:10C1D000F0B517480068016B3A22164B9C5E164D6D
:10C1E0002A681219154EB242154F03DAB94219D313
:10C1F000002318E001230E291F4600D800272D68D0
:10C200002C19B44200DC00233B400E22D2430C4FD9
:10C21000002B00D089184161C16AB94200D20F31A8
:10C220008160F0BD01230F22002BF3D1F3E7C0465C
:10C23000EC050020FC0C0020C41200206606000063
:10C24000F10F000006480068C16A0E2900D90F39B5
:10C25000026B81600E2A00D90F3A42617047C046D6
:10C26000EC05002006480068C26A06498A4200D2EE
:10C270000F32036B82608B4200D20F3343617047F1
:10C28000EC050020F10F00007047010180B500F0BF
:10C290007FF880BD70B501208403174D2C60174EC8
:10C2A000308917490880174800688047B0881649C8
:10C2B00008607089154A10601548036802261E43FD
:10C2C000066008681168884200DC08464021114A6F
:10C2D000515E88420AD310490A68101808600F4955
:10C2E0000968884205D90E48006880470A4800213D
:10C2F00001602C6170BDC04618080050D2130020A8
:10C30000C41200202C130020C8120020CC120020E0
:10C3100004000240FC0C0020841300206C04002068
:10C320004813002080B500F03BF80C2000F040F8E6
:10C330000B480C4901600C480068002800D080BD03
:10C340004120800009490A5A521C0A52084801211A
:10C35000016008480160084800680849086080BD1D
:10C360002C130020F9010020D0120020FC0C00202A
:10C37000D4120020C0120020B8120020680400204F
:10C3800080B5024800F01CF880BDC046BC0E0020FD
:10C3900008B4024B9C4608BC6047C04635320008D2
:10C3A00008B4024B9C4608BC6047C046C18C0008DC
:10C3B00008B4024B9C4608BC6047C0467D3D00085F
:10C3C00008B4024B9C4608BC6047C046ED9A000882
:10C3D00010B534480168062913D8C0467944097954
:10C3E00049008F440F1C031E032A3B002E490A6894
:10C3F0000021916051612D4A13685C1C1460E02B90
:10C400000BDA10BD28490A68002191605161274A62
:10C4100013685C1C1460002BF3D411601AE02A4AE4
:10C4200000E0284A204909688A604A611F490A6871
:10C43000531C0B60002A0BD510BD1B490968204A0C
:10C440008A604A6119490A68531C0B60012AD8DBCB
:10C4500000220A600168491C016010BD12490A6887
:10C46000002191605161114A13685C1C1460E02B3B
:10C47000C7DB0523036011600D4A13685C1C146060
:10C48000642BBEDB01601160092000F01FF8094831
:10C490000068002800D1084808490860092000F019
:10C4A0001DF810BD1C130020EC05002024130020F3
:10C4B0002013002008130020F90100202C13002075
:10C4C000FF0F0000FF0B0000FF07000008B4024B45
:10C4D0009C4608BC6047C0467D3D000808B4024B3E
:10C4E0009C4608BC6047C046653D0008040000004B
:10C4F000FFFFFFFFC0E0FFFFC0E0FFFFFFFFFFFF08
:10C500000024F40001000000FFFFFFFF0100000015
:10C51000FFFFFFFF01000000FFFFFFFF0100000021
:10C5200000B80B0002000000010000000400000041
:10C5300001000000020000000100000000000000F7
:10C5400002020000000000020202020201000000DC
:10C5500000000000000000000001010100010100D6
:10C5600001000202010100000000000000000000C4
:10C5700000000000000000000000000000000000BB
:10C5800000000000000000000000000000000000AB
:10C59000000000000000000000000000000000009B
:10C5A0000000000000000000000101010100010185
:10C5B0000000000101010100000000000000000077
:10C5C00000000000000000CDCDCDCDCDCDCDCDCD36
:10C5D000CDCDCDCDCDCDCDCDCDCDCDCDCDCDCDCD8B
:10C5E000CDCDCDCDCDCDCDCDCDCDCDCDCDCDCDCD7B
:10C5F000CDCDCDCDCDCDCDCDCDCDCDCDCDCDCDCD6B
:10C60000CDCDCDCDCDCDCDCDCDCDCDCDCDCDCDCD5A
:08E5C000CDCDCDCDCDCDCD00B8
:10E5C800206861680834002200E042540139FCD513
:02E5D80070478A
:10E5DA0020686168A2680C3401E08B5C8354013ABC
:04E5EA00FBD57047A6
:10E5EE00FFFFFFFFFFFFFFFFFFFFFFFFFFFFFFFF2D
:10E5FE00FFFFFFFFFFFFFFFFFFFFFFFFFFFFFFFF1D
:10E60E00FFFFFFFFFFFFFFFFFFFFFFFFFFFFFFFF0C
:10E61E00FFFFFFFFFFFFFFFFFFFFFFFFFFFFFFFFFC
:02FFFE00FFFF03
:020000040801F1
:10000000FFFFFFFFFFFFFFFFFFFFFFFFFFFFFFFF00
:10001000FFFFFFFFFFFFFFFFFFFFFFFFFFFFFFFFF0
:10002000FFFFFFFFFFFFFFFFFFFFFFFFFFFFFFFFE0
:10003000FFFFFFFFFFFFFFFFFFFFFFFFFFFFFFFFD0
:04EFFC00040CDD34F0
:040000050800ABEF55
:00000001FF
